:020000040000FA
:100000000002040000000000BC0200000A470000DB
:100010004847000086470000C4470000024800002F
:10002000BC020000BC0200004C380000BC02000012
:10003000BC020000F0300000283A0000BC020000C2
:10004000BC0200003C320000BC020000BC02000008
:10005000BC020000C6320000BC020000BC0200006E
:10006000243A0000BC020000BC020000BC020000F8
:10007000BC020000E0390000C4380000BC020000EF
:10008000BC020000BC0200002C3A0000BC020000D0
:10009000BC020000BC020000BC02000036390000B7
:1000A00014350000BC020000BC020000BC020000CD
:1000B000BC02000040320000303A0000BC020000E8
:1000C000BC020000BC020000BC020000BC02000038
:1000D000BC020000BC020000BC020000BC02000028
:1000E000BC020000BC020000BC020000BC02000018
:1000F000BC020000BC020000BC020000A8390000E5
:10010000C4390000BC020000BC020000FC39000041
:10011000BC020000BC020000BC020000BC020000E7
:10012000BC02000068370000DA370000343A0000F3
:100130003A3A0000BC020000BC020000BC02000011
:10014000BC020000BC020000BC020000BC020000B7
:10015000BC020000BC020000BC020000BC020000A7
:10016000BC020000BC020000BC020000BC02000097
:10017000BC020000BC020000BC020000BC02000087
:10018000BC020000BC020000BC020000BC02000077
:10019000BC020000BC020000BC020000BC02000067
:1001A000BC020000BC020000BC020000BC02000057
:1001B000BC020000BC020000BC020000BC02000047
:1001C000BC020000BC020000BC020000BC02000037
:1001D000BC020000BC020000BC020000BC02000027
:1001E000BC020000BC020000BC020000BC02000017
:1001F000BC020000BC020000BC020000BC02000007
:10020000FFFFFF00FFFFFF00BC02000040480000AE
:100210007E480000BC480000FA4800003849000051
:10022000BC020000BC0200004C380000BC02000010
:10023000BC020000F0300000283A0000BC020000C0
:10024000BC0200003C320000BC020000BC02000006
:10025000BC020000C6320000BC020000BC0200006C
:10026000243A0000BC020000BC020000BC020000F6
:10027000BC020000E0390000C4380000BC020000ED
:10028000BC020000BC0200002C3A0000BC020000CE
:10029000BC020000BC020000BC02000036390000B5
:1002A00014350000BC020000BC020000BC020000CB
:1002B000BC02000040320000303A0000BC020000E6
:1002C000BC020000BC020000BC020000BC02000036
:1002D000BC020000BC020000BC020000BC02000026
:1002E000BC020000BC020000BC020000BC02000016
:1002F000BC020000BC020000BC020000A8390000E3
:10030000C4390000BC020000BC020000FC3900003F
:10031000BC020000BC020000BC020000BC020000E5
:10032000BC02000068370000DA370000343A0000F1
:100330003A3A0000BC020000BC020000BC0200000F
:10034000BC020000BC020000BC020000BC020000B5
:10035000BC020000BC020000BC020000BC020000A5
:10036000BC020000BC020000BC020000BC02000095
:10037000BC020000BC020000BC020000BC02000085
:10038000BC020000BC020000BC020000BC02000075
:10039000BC020000BC020000BC020000BC02000065
:1003A000BC020000BC020000BC020000BC02000055
:1003B000BC020000BC020000BC020000BC02000045
:1003C000BC020000BC020000BC020000BC02000035
:1003D000BC020000BC020000BC020000BC02000025
:1003E000BC020000BC020000BC020000BC02000015
:1003F000BC020000BC020000BC020000BC02000005
:10040000AF2E21000E6F24000E01880000000000B6
:100410000C000700009A24000100200011000700D2
:10042000000020000000E000020032000000020096
:1004300000000000722D0200000000000040DA0001
:100440000000FE004440A900E01B20000000E00086
:100450000300320000002000A00188004440A800F2
:100460000000060091018800800078000000EB0089
:1004700015003700E280400032A0B4009101BA00BC
:10048000E280400032A0B4009102BA00E280400055
:1004900032A0B4000002EB00472BDE00F507B200EB
:1004A000602CE10004003A000059EB008301E900F0
:1004B000FDFF3E00040037006128E100010032002A
:1004C0000082EB00040007001101BA000200E00006
:1004D000E8FF3A00000006003159BA008301E90044
:1004E0000C0032002159BA008301E90008003200F3
:1004F0000400E00003003A00E280400032A0B400B3
:10050000F5FF370011D9BA008301E900FAFF3A007C
:100510008100E800E180400032A0B4000000060045
:10052000E81204000000000018120400000000009F
:100530003A120400000000005C12040000000000F9
:100540007E12040000000000AA1204000000000057
:10055000CA15040000000000CA19040000000000D1
:10056000321A0400000000009A1A04000000000083
:10057000021B0400000000000040DA000000FE0042
:100580000A00FA0080017800E20F500028003E00C7
:10059000B03C8200E10F50000800320080232000B0
:1005A0000000E00005003200042320002523200085
:1005B0004623200080017800040037000422200038
:1005C0002522200046222000832220001440900093
:1005D0000004E000040035008009EB0014409000A6
:1005E0000074A00010429800154090000028A3005D
:1005F00003003A00154090000024A00090429800AB
:100600008001EB0007003700154090000008A300B0
:10061000FDFF320063C078000000FB00000B780093
:100620008301E800828F5100F7FF3A00080037008D
:1006300030002000B0BF9F00C3BF9F00D1BF9F000C
:10064000E2BF9F006A80570000C0DA006FB99700D0
:10065000020078000080FA0000000600889FBE00BB
:100660008A9FBE008C1F7800C9000700D0003300AD
:1006700003866C006450E1002E0032006420E1002B
:10068000330032006150E1002F0032006120E100B0
:100690003100320085855500EB07B00009002000CD
:1006A00008042000050037000804440089844C0039
:1006B0000A0031000603430087834B00000153000A
:1006C00081815B00F8FF33000203BE000800A00038
:1006D0000804440089844C00F6FF3900C639DD0067
:1006E0008301730001003200130020008904D1004F
:1006F0000884D3000998A300050032000800A70071
:100700000300A0008904D1000884D3008B05E80011
:100710008904D1000884D3000001EB000281D200DB
:10072000B300070001F0A1000CF0A70001F0A00049
:10073000A80037006420E100AA0032000801BE00D2
:100740000200BE00F7FF37006120E100A500320083
:100750006000B800F3FF37000000200001F8270018
:10076000F0FF370003F0A200889FBE008A9FBE0002
:100770008C1F7800860007008D0033006450E10074
:100780004F0032006420E1005200320003826C000E
:1007900007003B000905D0000306D000820F54007B
:1007A0000C065D0002003900020032008901780069
:1007B000030678008582550004003D000003FD001B
:1007C0008103FD008502EA008B854200840F7200E0
:1007D00002003B0060001000E08018006011B800CB
:1007E0000005EB007A28E1000A00390006007800D5
:1007F000C75DDD00F707B200878075002D00370068
:10080000828171000A017800610560008180D10059
:100810000080D3008502E900F9FF3B000604400098
:100820008784480002003B0060041400E0841C0040
:100830000988A300070032008A817100828171005B
:10084000610164008904D1000884D3008B05E800AD
:10085000170037000978A30013003A000B00E000EE
:10086000130034008B05E9000804440089844C001F
:100870000A4474000978A3000D003A000B00E00060
:10088000070034008B05E9000804440089844C000B
:1008900001003A000B0020000978A300F7FF3200A6
:1008A0000001EB0002003700828171000A0178002C
:1008B0004F0007000CF0A70001F0A0004500370032
:1008C0006420E10002003A00838F6C004500330091
:1008D0000801BE000200BE003E003700889FBE0037
:1008E0008A9FBE00010578000100E0000400350089
:1008F00008003C000000E000200032000500370046
:1009000060001000E080180002003B0001F02C00A5
:100910001A0037000004BE006011B8006B09200007
:100920000982CF00020039000882CF000441B000E4
:10093000694252000E00320008003B0082817100C3
:10094000610164008904D1000884D3008B05E800AC
:100950000442E800F9FF3A000500370008044400AB
:1009600089844C008B05E9000442E900FBFF3A0052
:100970001F0007000AF0A70001F0A0004F05BE000D
:100980004F04BE0000000600F4FF2F003E003700B9
:100990000004BE00570007000003BE000405BE00AF
:1009A0000200BE0053000700844F750000000600DF
:1009B0000200BE006450E100050036006420E10042
:1009C000020036000968A30001003A000800BE00DA
:1009D0000160A0004F0678004F05BE004F04BE0026
:1009E00000000600F0FF2F00F1FF2700F9FF37009D
:1009F00081002000618055000B003D000B002000AD
:100A000061FE2F000100E1001D00340082817100B1
:100A1000610164008904D1000884D3000000E8006B
:100A2000FAFF3A00710020006100640003007000CA
:100A3000020060000900320061044400E0844C00C0
:100A40000988A500050032008B05E8006808E10070
:100A500002003A008904D1000884D300F20F20007C
:100A60000258E10005003D00C75DDD00F907B20056
:100A70008980750008007800000006000BF8270048
:100A80008B00780000000500889FBE008A9FBE0092
:100A9000841F7800BEFF07004F007800110033006C
:100AA000F0FF2F00838F6C0006003B0004056500FB
:100AB0000A00A7000800370009F0A6001000200077
:100AC00008003700820F5400838F5C000300390058
:100AD0001000200001003E000000200009F0A700E7
:100AE0000000EA004F05BE004F04BE000000E00019
:100AF00000000600C70ADE00F107B200F50FB200E1
:100B000008003200E1CF4200020032000170A00074
:100B100024000500810F7000010032000408050068
:100B200044000500810F700002003A001400050027
:100B30008502E9000000400081C04800FCFF3B0046
:100B40000170A00024000500881F780000047800D0
:100B50005001BE004000BE000400400085804800F7
:100B60000601490087814900009CBE000294BE0036
:100B70000400E1000588E1000690E1000798E1002B
:100B800002003100680044001008E8004F047800BB
:100B900000000600F4874700889FBE008A9FBE00C1
:100BA0008C9FBE008E1F78000205BE000004BE00B0
:100BB000D4B79F00E5B79F00F6B79F0087BF9F009F
:100BC0000000EB00C0B79F00B0B79F00A0B79F0028
:100BD00090B79F0080B79F000D042000BFB0970022
:100BE0004FB09700000140000000E0000F003D0002
:100BF0004F08DE0000007100C0B79F009E00070094
:100C000001003D0012002000A100070001003D008E
:100C100012002000A6000700B1000700B600070080
:100C20000F004000C8FF0700220037004F08DE0019
:100C300000067100CCB79F008F00070001003D0047
:100C4000120020009200070001003D001200200069
:100C500097000700A20007000FB297009FB297000D
:100C60002FB39700BFB39700A90007000000520000
:100C700081805A0002015B0083815B0080B79F0086
:100C800091B79F00A2B79F00B3B79F000007EB008A
:100C90009F0007000020E10001A8E10002B0E10090
:100CA00003B8E100010031001E0020000E005600D4
:100CB000C0B79F004FB297000400E0000700350066
:100CC00010002000010020006011B800080470002E
:100CD000898470000A0571008B8571008D06E9001A
:100CE000BEFF3A000400E00003003D008200070060
:100CF0000F00400094FF07004FA897000000E0009D
:100D000004003A000FB497009FB497002FB59700E6
:100D1000BFB59700940007004F0778004F06BE004C
:100D20004F05BE004F04BE004F01B1000000060099
:100D3000881F780018002000881F780095FF0700A2
:100D40008F87E9004F04780000000600801FEB0049
:100D500090FF07008F87E90000000600889FBE0013
:100D60008A9FBE008C1F78006E00070007003D00C0
:100D700073000700E00F5B00E08F5B0007003D00A1
:100D8000320007000006EB000400370034000700C3
:100D900002003D002A0007001C002000720007002E
:100DA000E3FF07000203BE000002BE000C00E000EB
:100DB00001003200220007000400BE000601BE0050
:100DC0004F0678004F05BE004F04BE00000006002D
:100DD000889FBE008A9FBE008C1F780051000700CC
:100DE00005003D0056000700E00F5B00E08F5B0050
:100DF00006003D00040037001900070003003D0015
:100E00006000B8006011B80010000700560007002D
:100E1000CEFF07000203BE000002BE000C00E0008F
:100E200001003200060007000400BE000601BE00FB
:100E30004F0678004F05BE004F04BE0000000600BC
:100E40006000B8006011B8000000370004025000D4
:100E50008582580006035900878359000000060068
:100E60000006EB00E00F5200E08F5A00E00F5B003D
:100E7000E08F5B00000006000180400090B79F00FB
:100E80000001EB008FB097000100E00000000600B9
:100E90000200700090B79F000180400080B79F0063
:100EA0000001EB00FFA897000100E0000000060031
:100EB0000200700080B79F00018040006FAA970079
:100EC000CF20DE0001007000F0AF9F00040242005E
:100ED000250007004F18DE00000272000000060027
:100EE000E4AF9F000804440089844C000A054D00CB
:100EF0008B854D00000006003FB29700CFB29700EF
:100F00005FB39700EFB3970000FE2F0000000600CC
:100F10003FB09700CFB097005FB19700EFB1970057
:100F2000000006000205BE000004BE00E00F5000F5
:100F3000E08F5800E00F5900E08F590000000600D4
:100F40006000B8006011B80008045000898458009F
:100F50000A0559008B8559001C002000E00F520043
:100F6000E08F5A00000006000800BE000A01BE0023
:100F7000000006000C00FA00889FBE000004780004
:100F8000CFB09700F0FF2700D0BF9F008004EB0098
:100F900099BF9F0088BF9F00A8BF9F00200C200022
:100FA000B0BF9F0078815700708057005400070041
:100FB0000FB89700094878000FB897000804500050
:100FC000080078004F04BE000080FA000000060010
:100FD0000001780000C2B300010037000201E80000
:100FE0009240780080CF5000FCFF3200E9CF5000E3
:100FF000FAFF3200D0C2B30080CF500003003A00A5
:101000000201E80014C0B300050037000042EB0005
:10101000B0C2B30080CF500001003A000201E800E6
:101020008000EB0005FD2F00040037006A08B900BE
:1010300000804100850040000201E8009201FB00B1
:1010400005804100E90F5000F8FF36000404E0007D
:10105000010032008100EA00010078000000060073
:10106000810178000002EB000B003700E4407800BB
:101070000104E000030032000402E80093CF5000B6
:10108000040032008180FB001380FB0000805000D0
:10109000000006008301E800820F5200F3FF3A00CF
:1010A000000005000003780080027800020278004A
:1010B0008001EB00080037000402E90063C07800FB
:1010C000805A78008301E8000004E00002003A0042
:1010D0008000EB0006003700828F5100F6FF3A00D7
:1010E000FBFF37000040EB0080F07A008100E80051
:1010F000848F5000FBFF3A000600780000000600D5
:10110000FE874700889FBE008A9FBE008C9FBE005E
:101110008E1F7800F0B79F000107780082BF9F0004
:101120000000EB00A0B79F009F0237008006EB0095
:1011300050C2B30080CF5000090032000100FB0014
:10114000FFB09700A3020700E10F400096023200B3
:10115000AFB097008100E800A1B79F00920237006E
:101160009E407800D0C2B30080CF50000C00320007
:1011700007003C006D40500080CF50000A00320054
:101180006B40400080CF50000E003A00080037004E
:1011900000C3B30080CF50000A003A0006003700B9
:1011A0000D30A000050037000D00A000030037003F
:1011B0000D10A000010037000D20A0000E07E80070
:1011C000E7FF37000D18A300010032000D00A10059
:1011D0000D38A300010032000D20A1000100FB002A
:1011E00002FD2F0002004000E90F50000E003E00FB
:1011F0000002EB00C4B79F0082017800CFB29700D5
:101200006A28B9001E01FB000001410003014100F2
:10121000C2B79F005E00FB0003004000E90F5000D2
:101220000B003E00F5FF37000006EB00CCB79F0037
:10123000A0C2B30080CF500005003A000FB897005D
:10124000C000780080BF9F00C1B79F000E07E80074
:101250000001EB00B2B79F00E0C2B3009E4F100048
:1012600018003A000DE0A0008E00E8006440500035
:10127000914F100002003200010778000C00370087
:101280000FBA9700C402780084BF9F00B5B79F00D3
:101290000E87E8000B0037003FB697006A60B90080
:1012A0000000410003004000B0B79F000E07E800B7
:1012B0001E01FB0003FD2F0003004100E90F500059
:1012C000F5FF3600BE407800E1D79F00C0C6B300EE
:1012D00080CF5000220032000F003C0069405000D7
:1012E00080CF50007700320004003C000104E00091
:1012F000310232006B4050000F00370040C6B3008F
:1013000080CF5000930032006540400080CF5000F5
:101310008B003A008F00370030C7B30080CF5000F9
:101320001A00320007003C006440500080CF50009B
:10133000110032000040E80080CF500080003A00E9
:101340000F00370050C7B30080CF5000800032003C
:101350006340400080CF500079003A000900370018
:10136000000028000D48A30001003A000001200001
:1013700080867600D3FF37000D60A000750037002F
:101380000D50A0000D70A000720037008FB89700BC
:101390004100780081BF9F00000478000000E00059
:1013A00001003A00087424008004EB0001003700BB
:1013B0008104E80089007800088044001004E000FF
:1013C000FBFF3A003FB197000200E000030032004B
:1013D000890F510001003100820478000002EB0007
:1013E000E4AF9F00CFB29700898F52000200360011
:1013F00009805200E0AF9F004368DE00E106600014
:101400001B003A000D06780009003700FFB0970076
:1014100000022000EF010700E10F4000030032004E
:101420002FB097000000E800A0B79F000C06E8006E
:10143000EFA89700810F5600F4FF3A000081EB00FF
:10144000E2AF9F000A003700880078003100FB00FF
:1014500001047800FFB09700DE010700E10F4000B3
:10146000030032002FB297000402E800A4B79F00E7
:101470000900E90080047800E10F4000F2FF3A0023
:101480000006EB000D00E0000A003A00C60137003C
:10149000FFB0970000022000CE010700E10F4000DE
:1014A00003003200AFB297008502E800A5B79F00A5
:1014B0000C06E8006FA89700800F5600F4FF3A0072
:1014C000B90137008FB897004100780081BF9F00B5
:1014D000CF80DE0001017800820178000205BE00A5
:1014E0000004BE000203BE000002BE004822DE006F
:1014F000482EDD0004027600E4D79F000D48A300CB
:101500000A0032000404E00008003200E14F42000B
:101510000600320071FD2F0001804700044878006A
:10152000184098002900200002003700F0D79F00E3
:101530001900200072FD2F0002844700A1FF370030
:1015400064FD2F0004844700190020009DFF370030
:101550000D0CB3000D007800000CB20028003A001A
:101560000D00E00005003D008FBA97004505BE0064
:101570004504BE0085BF9F00140037000D48A3003E
:101580000B0032000FBE97004C00BE008CBF9F00C6
:101590004F89DE00CF91DE000002BE00020378001A
:1015A000820378000605BE000404BE000700370071
:1015B0008FB897004100780081BF9F000004780039
:1015C000CFC4DE00090578008A057800E00F5400DA
:1015D000E08F5C00E00F5D00E08F5D001F003D00CC
:1015E0003D00B3006000B8006011B800080450006E
:1015F000898458000A0559008B8559001700370067
:101600000D00E00005003D000FB997004205BE0047
:101610004204BE0082BF9F00100037000D48A300A7
:10162000070032000FBA97004400BE0084BF9F003D
:101630006011B8000205BE000004BE0007003700BC
:101640008FBA97004500780085BF9F00000478009E
:10165000090020000A0020000B0020003FB6970080
:101660000C00E00007003A00E00F5400E08F5C003F
:10167000E00F5D00E08F5D0002003A0010002000E6
:10168000B0B79F008D007800010CB200E1B79F0059
:1016900000042000808F50003000320003003C0026
:1016A0000100E00008003200400037000008200080
:1016B0006FB19700800F510014003200000C200021
:1016C000800F510039003A0014C0B300A5E4200097
:1016D0000B0037000400FB004300DD000500400064
:1016E0005001BE004000BE000040E10001C8E10022
:1016F00002D0E10003D8E1002B0039000442E800E9
:10170000F44F5200F3FF3A00270037000001200099
:10171000010020006011B80014C0B3000040E100D7
:1017200001C8E10002D0E10003D8E1001E00390049
:10173000450020000000D0008180D2000281D2004C
:101740008381D2008502E900FAFF3A000442E800F2
:10175000F04F5200F1FF3A001300370080002000E4
:10176000010020006011B80014C0B3000040E10087
:1017700001C8E10002D0E10003D8E1000A0039000D
:101780003C0020000000D0008180D2000281D20005
:101790008381D2000C06E900FAFF3A000442E80017
:1017A000F54F5200F1FF3A00E4D79F00EFD09700C9
:1017B0000100FB003FB19700820F500002003D0086
:1017C000E2D79F00040037003FB29700800F52001D
:1017D00001003D00B0B79F00CFB297000500E000C8
:1017E0000400320063806600020032008502E900D6
:1017F000C5B79F000DE8A3000B0032004FB697005D
:101800003FB09700800F560003003C008000EB00C3
:10181000C1B79F00040037004FB197003FB2970057
:1018200004015100C2B79F00EFD297000500FB00F2
:101830000006EB00DCAF9F00CFB09700808F500018
:101840000200340000805000D0AF9F000D28A3009C
:1018500037003200E18066000D18A3000C00320052
:10186000D00220000100E00001003A000080E90001
:10187000FFB09700D7000700E10F40000E003200D4
:101880002FB197000201E800A2B79F000A003700BD
:101890000100E00008003200FFB0970000022000C5
:1018A000CC000700E10F4000030032002FB2970088
:1018B0000402E800A4B79F00DFAA97000500E0003B
:1018C0000F0032000006EB00FFB09700000320007D
:1018D000C0000700E10F4000030032002FB0970066
:1018E0000000E800A0B79F000C06E800DFA8970002
:1018F000810F5600F4FF3A000001EB00D2AF9F00C9
:101900003FB29700C320DD0020E42000808040002B
:1019100091B79F004220DD006400500080B79F0017
:101920006320B900F0AF9F006306500084003700C9
:10193000DFAA97000500E000110032006880660011
:101940000F003A0000067800FFB097000002200068
:10195000A0000700E10F4000030032002FB0970005
:101960000000E800A0B79F000C06E800DFA8970081
:10197000810F5600F4FF3A000001EB00D2AF9F0048
:10198000E18066000D18A3000C003200D002200098
:101990000100E00001003A000080E900FFB097007C
:1019A0008C000700E10F4000D5FF32002FB29700F6
:1019B0000402E800A4B79F00D1FF37000100E00057
:1019C000CFFF3200FFB09700000220008100070027
:1019D000E10F4000CAFF3200AFB297008502E80075
:1019E000A5B79F00C6FF370000042000EFB09700A6
:1019F000808F50003100320003003C000100E00005
:101A0000080032003E003700000820006FB1970048
:101A1000800F510011003200000C2000800F510097
:101A200037003A001FB097003002BE002003BE000E
:101A30000800BE000A01BE00BDFC0700A400200093
:101A4000050020006033B800C0FC070004C3B300E9
:101A500004424000E4D79F00290037007574240039
:101A6000D5B79F000D58A30002003A0080752400EE
:101A7000D0B79F0014002000050020006033B8009C
:101A80008FB097008100E900050033000402D00008
:101A90008582D2000683D2008783D200F9FF370007
:101AA0000800BE000A01BE00A1FC07006F00600034
:101AB0005FB19700624078001000370014002000EA
:101AC000050020006033B8000C0078000000E90039
:101AD000050033000402D0008582D2000683D200C4
:101AE0008783D200F9FF37000800BE000A01BE005C
:101AF0008FFC0700674060000043B000E0D79F0004
:101B0000EFD097000100FB00FFB097003100070005
:101B1000E10F4000030032002FB197000201E800FE
:101B2000A2B79F001FB297006802520094B79F00AF
:101B30008FB29700E482520085B79F00630656007B
:101B4000D0FF2F003FB197000090B9007FAA970007
:101B50000000420063005000800F5600A2FF3A00D0
:101B60000D38A30010003200DFAA97000500E00046
:101B70000D0034000006EB00FFB0970000022000CB
:101B800014000700E10F4000030032002FB097005F
:101B90000000E800A0B79F000C06E800DFA897004F
:101BA000810F5600F4FF3A00BE407800E1D79F0055
:101BB0000104E0005DFD3A002FB097004F07780068
:101BC0004F06BE004F05BE004F04BE00EF01B1003E
:101BD00000000600889FBE00000178000104780024
:101BE000B10090000118A3003D0032000198A3004D
:101BF00003003A00180090000000E00038003A00AE
:101C00000190A0003104980082047800F90FB2001E
:101C1000180090000000E00002003A002800900048
:101C2000000C7800EA8F540006003A00380090005B
:101C30000078A30003003A0088007800D00020005C
:101C4000E4FF07009800900058009000808F50003B
:101C50000B0032000100E800100498001800780022
:101C600009587800000C780011C0B30040792400B6
:101C700001487800EA8F540006003200190037004E
:101C80008800780009407800190007008004780077
:101C900014003700380090000088A30011003200C3
:101CA00018019000A80090004800900034FA070046
:101CB00098009000810F500004003200380090001E
:101CC0000003B300300498008084EB000000EB00B8
:101CD0001004980028009000000C780001003700E4
:101CE0008084EB00090078004F04BE00000006006D
:101CF0000200FA00889FBE00A0FF9F000104780048
:101D0000B1009000810478000904B20002003200A2
:101D10000000FB00360037000118A30005003A0060
:101D20000103B30031049800190498000080EB000F
:101D30002F003700580090000000E00006003A0035
:101D40004800900012002000E68057000CFA0700BF
:101D50001904980024003700280090000000E000DB
:101D600008003A000079240020049800000C780054
:101D70002000200050049800100498000130A000BA
:101D80003104980018019000A800900048009000CD
:101D9000FBF9070028009000000C78000080EB00A1
:101DA0001004980018007800AFF8970001587800E8
:101DB000000C78002FF89700EA4F50000A003A0014
:101DC000380090000088A30007003200180190003E
:101DD000A800900048009000E9F907001904980055
:101DE000A8009000010C7800AFF897000100FB00FC
:101DF0004F04BE000080FA0000000600636C000083
:101E000074000000737400006C0000007366000032
:101E100061000000737300006C000000736F00002D
:101E20006C00000073610000640000007263000039
:101E300066000000727400006C0000007266000012
:101E400061000000727300006C000000726F0000FF
:101E50006C000000434C000054000000535400008C
:101E60004C000000534600004100000053530000A6
:101E70004C000000534F00004C0000005341000094
:101E8000440000002530000034580000000D000020
:101E90000D2000004C440000435B00002532000090
:101EA000645D00003A0000000D0000000D3E0000DF
:101EB0003E20000041470000565F000056330000FE
:101EC00035300000204C000049460000542000003E
:101ED00044520000495600004552000028320000DC
:101EE00030320000342E0000313100002E3200006C
:101EF000362900003C3C0000000D0000204C000092
:101F000044430000204100004444000052200000EF
:101F10003D2000000025000034640000000D00009A
:101F2000204F000043520000202000004C450000DC
:101F3000562000003D200000000D0000205400004D
:101F4000494D0000452000004C4D00005420000089
:101F50003D200000000D000020460000415300001D
:101F60005420000053500000442000003D20000099
:101F7000000D0000205300004C4F000057200000CF
:101F800053500000442000003D200000000D0000E0
:101F90000D0D0000000D0000206300006F6D0000BB
:101FA0006D6100006E640000206E00006F74000020
:101FB000206600006F7500006E6400002E2E000089
:101FC0002E210000000200002530000034640000D3
:101FD000414300004B250000303400006400000045
:101FE000022500003034000064530000544C00000F
:101FF000253000003464000000020000253000009D
:1020000034640000534600004125000030340000D5
:10201000640000000225000030340000645300001A
:10202000534C000025300000346400000002000022
:102030002530000034640000534F00004C250000A0
:1020400030340000640000002530000034640000DB
:10205000000000000D2000005F460000414C000021
:1020600054410000204900006E74000065720000B9
:1020700072750000707400002E2E00002E2E0000DD
:102080002E210000000D0000205F000046410000EE
:102090004C54000042200000496E000074650000AE
:1020A0007272000075700000742E00002E2E000069
:1020B0002E2E0000210000004C44000043200000B0
:1020C000494E0000543100002E2E00002E21000049
:1020D000004C000044430000204900004E54000022
:1020E000322E00002E2E0000210000004C44000083
:1020F00043200000494E0000543300002E2E000003
:102100002E210000004C0000444300002049000044
:102110004E540000342E00002E2E0000210000003E
:10212000434E0000492E00002E2E0000210000002A
:102130004C49000046540000204400005249000071
:1021400056450000522000004C6F00006164000002
:102150002044000065660000617500006C7400009A
:1021600020560000616C0000756500002E2E0000F6
:102170002E2E00002100000080407800910A070008
:10218000FEFF32000100FB00201188000000060065
:10219000804078008E0A0700FEFF32000100FB003D
:1021A000A0118800000006001F0A07000700360083
:1021B000F0CBB30000404100F10F2000E54F50008C
:1021C00003003E0090CCB300004041008080FB0043
:1021D0000100780000000600130A07000600360020
:1021E000F10F200000C4B300804F510003003600FF
:1021F00090CCB300004041008080FB00F4FF37002A
:10220000E94F500003003E000043B0000080FB0097
:10221000000006007043B000FCFF37001E00FA000B
:10222000889FBE00000478006C0A0700640040002C
:102230008286200060007900E404500067005000AE
:10224000FB0F500032003E000900E0003400320075
:102250001841780001CEB30001404100A5C5B3008C
:10226000854F50002A003E008001EB0003027800F9
:102270000900E900630060000E0032000202FB006A
:102280001300200063417C008140410085CF500055
:102290001F003E00E10F500006003200E20F500028
:1022A00002003200F909070019003E00F709070093
:1022B00017003E00740A07008302E80085017800D9
:1022C000858F540017003200F209070010003E000D
:1022D0006D0A07008501E800EE0907000C003E00CA
:1022E000690A07008581E80063417C00874041005E
:1022F00086CF500006003E00630A0700E3814200DB
:1023000063417C008740410086CF5000E9FF3600E2
:102310000000EB004F04BE000080FA000000060041
:1023200009027800841F780020F42800801F7800BC
:10233000A0FD2F000F0040000EFB07008880440026
:10234000E48757000FE09700914F500006003200DD
:102350000041EB000280FB004F04BE000080FA0049
:1023600000000600EEFF37009140900012C0B3005D
:102370001FE09700814F5000F6FF32000041EB0054
:10238000F4FF37000A00FA00889FBE0000047800BE
:1023900081447800104078008000EB000004E000E9
:1023A00010003A00811F780020F42800801F780078
:1023B00072805700EFFA07000FF09700004C78008A
:1023C0001FF0970010449800294498000040EB004B
:1023D00030449800E48757004F04BE000080FA00A4
:1023E000000006000000FB0080804000584078009C
:1023F0000004E000EBFF32000000FB0080804000A2
:10240000584078000004E000F6FF3A00E5FF37008E
:1024100010C0B30046E8B7000040EB0048E8B70042
:1024200047E8B70050C0B30049E8B7000000060015
:102430000600FA00ED09070066805700E4FA07007D
:10244000F509070003003600020078000080FA005A
:1024500000000600116E8800116E800080012000CF
:10246000520B0700100020000080FA000000060058
:10247000F8FF37000600FA00DC0907006680570005
:10248000D3FA0700E90907000300360003007800CB
:102490000080FA0000000600F26D880082007800DB
:1024A00060012000410B0700100020000080FA00AE
:1024B00000000600F8FF37000600FA00CB0907000D
:1024C00066805700C2FA0700D809070003003600EB
:1024D000030078000080FA0000000600026E880009
:1024E0008200780040012000300B0700100020001F
:1024F0000080FA0000000600F8FF37000600FA002E
:10250000BA09070066805700B1FA0700C209070040
:1025100003003600020078000080FA000000060088
:10252000216E8800216E8000200120001F0B070013
:10253000206E8000120020000000E000F5FF3A004D
:10254000A06A8800020078000080FA0000000600FF
:10255000F3FF37001E00FA0090407800A1E79F00CB
:1025600090409000B1E79F00A0409000C1E79F001D
:1025700030409000D0E79F000040EB00E0E79F0074
:102580007E80570092FA0700000178008000E90081
:102590008001EB0020062000808F500009003E00E3
:1025A000306E800013002000800F510005003200C3
:1025B000326E8800316E800000012000FB0A0700A7
:1025C00013002000030078000080FA0000000600DD
:1025D000100005000600FA009A0907008286200014
:1025E0000000410000489000A0FF9F0099090700EB
:1025F00010489000B0FF9F00960907002048900007
:10260000C0FF9F00A9090700000141003249900066
:10261000D2FF9F000040EB00E0FF9F006680570064
:102620006BFA070080007800306E800080806800C0
:102630000100EA00010070004F00DE0061001000A0
:102640000080FA0000000600C82DA9007D090700DF
:1026500064004000868620000001EB0002307B0011
:102660007F090700124098007D09070002487800A2
:10267000824378008A090700924098000201E8002E
:102680007A0907000201E800780907007A090700C3
:1026900006090700E780400004090700E8804000C1
:1026A00002090700E980400000090700EA804000B5
:1026B000FE080700EB8040008680400097409800AD
:1026C00066014000FE0F5100EFFF3A006968EC0020
:1026D00069C8BF00FD4F5000010036006968EF0077
:1026E00092862000124178008041EB0044022000D5
:1026F00006090700010032000A0907000D0907005A
:10270000010036000041EB008341E800FF080700AC
:1027100016003A0007090700010036000041EB00EF
:10272000FA08070013003A0002090700010036000A
:102730000041EB00F508070010003A00FD08070013
:10274000010036000041EB00F00807000D003A00E0
:10275000F8080700010036000041EB00E4C1410029
:10276000FECF5100E2FF3A0000000600ED0807002E
:10277000E8FF3700EB080700EBFF3700E908070028
:10278000EEFF3700E7080700F1FF3700304178001F
:1027900080017800A508070013003E008040780003
:1027A000440ADD0013417800A008070003003E0042
:1027B000804078000140420094FE3700F0CBB30027
:1027C0000040410080C0EB00E54F5000F9FF3E00A3
:1027D00090CCB30080404100014042000080FB00EB
:1027E00000000600F5FF3700F0CBB30000404100C9
:1027F00080C0EB00E54F5000E9FF3E0090CCB300F5
:1028000080404100E6FF37000001780090407800EA
:102810000104E00005003A0000000600E908070096
:10282000FEFF3200C6080700FBFF32000201E8008D
:10283000E4080700F9FF3200FAFF370000017800D2
:10284000D442E20009003500904078000104E00025
:10285000050032000201E800DA080700FEFF32003E
:10286000B7080700FBFF3A00000006000000060062
:102870001400FA00881F780000047800D442E200B7
:1028800003003D004F0478000080FA0000000600BD
:10289000306E8000801F780070F42800801F780060
:1028A0007A805700B3F90700EFE09700E4875700FC
:1028B0000104E0000A003200768157000201E800BE
:1028C00023C2BF000008A300FDFF32000100FB008F
:1028D00020118800924078000104E000F7FF3A00E0
:1028E000984078000104E000E6FF32000804E800A8
:1028F00023C2BF000008A300FDFF32000100FB005F
:1029000020118800F6FF37003200FA0042F5280057
:10291000D1C0B3000201E800AA080700FEFF3200A0
:1029200087080700FBFF3A0062F52800D1C0B3001A
:102930000201E800A3080700FEFF3200800807003C
:10294000FBFF3A0042F52800D1C0B3000201E800C5
:102950009C080700FEFF320079080700FBFF3A00E1
:10296000D2F72800D1C0B3000201E80095080700A3
:10297000FEFF320072080700FBFF3A00306E800055
:10298000801F7800B0F82800801F7800A0FC2F007E
:102990000F00400077F90700AFC89700E4875700A1
:1029A0000104E00007003200E2FC2F000F014100AB
:1029B0000201E80083080700FEFF320060080700FC
:1029C000FBFF3A0042F52800D1C0B3000201E80045
:1029D0007C080700FEFF320059080700FBFF3A00A1
:1029E000F2F82800D1C0B3000201E8007508070022
:1029F000FEFF320052080700FBFF3A00206E800005
:102A0000801F7800B0F82800801F7800A0FC2F00FD
:102A10000F00400057F90700AFC89700E487570040
:102A20000104E00007003200E2FC2F000F0141002A
:102A30000201E80063080700FEFF320040080700BB
:102A4000FBFF3A00D2F92800D1C0B3000201E80030
:102A50005C080700FEFF320039080700FBFF3A0060
:102A6000106E8000801F7800B0F82800801F78006A
:102A7000A0FC2F000F0040003EF90700AFC89700F0
:102A8000E48757000104E00007003200E2FC2F0059
:102A90000F0141000201E8004A080700FEFF320072
:102AA00027080700FBFF3A00B2FA2800D1C0B300A4
:102AB0000201E80043080700FEFF3200200807007B
:102AC000FBFF3A00F06D8000801F7800B0F828000E
:102AD000801F7800A0FC2F000F00400025F90700A0
:102AE000AFC89700E48757000104E00007003200F8
:102AF000E2FC2F000F0141000201E800310807004D
:102B0000FEFF32000E080700FBFF3A0092FB280090
:102B1000D1C0B3000201E8002A080700FEFF32001E
:102B200007080700FBFF3A00006E8000801F780056
:102B3000B0F82800801F7800A0FC2F000F00400094
:102B40000CF90700AFC89700E48757000104E000C4
:102B500007003200E2FC2F000F0141000201E800F3
:102B600018080700FEFF3200F5070700FBFF3A00D8
:102B700072FC2800D1C0B3000201E8001108070070
:102B8000FEFF3200EE070700FBFF3A000080FA006C
:102B9000000006005CFF070000000500000178004F
:102BA000904078000104E00005003A0000000600B3
:102BB00007080700FEFF3200E6070700FBFF3200B0
:102BC0000201E80002080700F9FF3200FAFF3700AF
:102BD000A1842000914078000104E0000A00320046
:102BE0000001EB00B3842000F9070700FEFF32006C
:102BF0000100FB00A0118800E2C079000201E8009A
:102C00000104E000F8FF3A0049C8BF0003003200A9
:102C10004968ED004868EF000000060046E8B7008C
:102C20004868EF0000000600FCFF37004200FA0091
:102C3000889FBE008A9FBE00CB07070089862000C0
:102C40000080440000489000E0779F00CA0707001A
:102C500010489000F0779F00C707070020489000B9
:102C6000807F9F00C407070030489000907F9F003E
:102C70000040EB00A07F9F0060FB2F000F00400092
:102C8000D3F80700316E8000810F5000040032003D
:102C90004F05BE004F04BE000080FA000000060091
:102CA00069C8BF000080FB000880B90000804400B4
:102CB000C048900020C7B30080CF50008B00320086
:102CC00069C8BF000080FB000880B9000080440094
:102CD000C048900030C7B30080CF5000F7003200EA
:102CE00069C8BF000080FB000880B9000080440074
:102CF000C048900030C6B30080CF5000230032009F
:102D000069C8BF000080FB000880B9000080440053
:102D1000C048900030C4B30080CF50001B00320088
:102D2000D442E200DAFF350050FC2F000084470057
:102D3000316E8000811F780070F42800801F7800B9
:102D4000080078008BF8070098407800E487570067
:102D50000104E00076013A00B2FC2800D1C0B300C3
:102D60000201E80023C2BF000008A300FDFF3200FB
:102D70000100FB0020118800924078000104E0006F
:102D8000C3FF32000201E800F6FF370069C8BF0048
:102D90000080FB00480220000880B9008A862000DD
:102DA00000804400ED004000E40DEC002200200013
:102DB000ABF807000004E000B5FF3A0069C8BF00A7
:102DC0000080FB000880B90064004000E0007D0046
:102DD000406F8000808F5000ADFF3A0069C8BF008F
:102DE0000080FB000880B900000045006F00400033
:102DF000316F800001000100E14F5000A4FF3A0054
:102E000069C8BF008080FB00400220000088B90034
:102E10006600400009044000306E800001418000DF
:102E200099FD2F0089844700801F7800811F78005A
:102E300031FE2800811F7800090078004DF8070056
:102E4000E60044006C8044003200200095F8070042
:102E50000040EB00A0E79F004FD09700E6875700A7
:102E60000004E0003E013A000904E8008000EB00A5
:102E7000811F780020F42800801F780071FB2F004C
:102E8000018047003BF807001F789700004C78004E
:102E9000AF7897001144980030C0B30020449800E8
:102EA0000040EB0030449800F0E79F009940780024
:102EB000E48757000104E00075FF32000901780043
:102EC0000201E80023C2BF000008A300FDFF32009A
:102ED0000100FB0020118800924078000104E0000E
:102EE0006BFF32000201E800F6FF370069C8BF003F
:102EF0000080FB000880B90000804400ED00400025
:102F0000080EEC002200200055F807000004E00045
:102F100009003A0069C8BF000080FB000880B900C2
:102F200064004000E0807C000001EB0060708000E5
:102F3000808F50005000320069C8BF000080FB0045
:102F4000480220000880B90000804400ED004000E5
:102F50000E0EEC002200200041F807000004E00003
:102F600009003A0069C8BF000080FB000880B90072
:102F700064004000E0807C0012002000907080001F
:102F8000808F50003C00320069C8BF000080FB0009
:102F9000480220000880B90000804400ED00400095
:102FA000140EEC00220020002DF807000004E000C1
:102FB00009003A0069C8BF000080FB000880B90022
:102FC00064004000E0807C0022002000C07080008F
:102FD000808F50002800320069C8BF000080FB00CD
:102FE000480220000880B90000804400ED00400045
:102FF0001A0EEC002200200019F807000004E0007F
:1030000009003A0069C8BF000080FB000880B900D1
:1030100064004000E0807C0032002000F0708000FE
:10302000808F50001400320069C8BF000080FB0090
:10303000480220000880B90000804400ED004000F4
:10304000200EEC002200200005F807000004E0003C
:103050000FFF3A0069C8BF000080FB000880B9007C
:1030600064004000E0807C0020718000808F500070
:1030700007FF3A004200200069C8BF008080FB00C3
:10308000400220000088B900808144006610B90029
:103090000080E800EF81410082E02000E00079003C
:1030A00003007800010001004F05BE004F04BE0080
:1030B0000080FA0000000600F9FE370069C8BF0072
:1030C0000080FB000880B90000804400ED00400053
:1030D000EA0DEC0022002000E1F707000004E00008
:1030E0004200320069C8BF000080FB004802200097
:1030F0000880B90000804400ED004000F00DEC00B5
:1031000022002000D6F707000004E0004B00320048
:1031100069C8BF000080FB00480220000880B90099
:1031200000804400ED004000F60DEC00220020007D
:10313000CBF707000004E0005400320069C8BF006C
:103140000080FB00480220000880B9000080440095
:10315000ED004000FC0DEC0022002000C0F707004D
:103160000004E0005D00320069C8BF000080FB0081
:10317000480220000880B90000804400ED004000B3
:10318000020EEC0022002000B5F707000004E0006A
:10319000BFFE3A0069C8BF000080FB000880B9008C
:1031A00064004000E0807C0030708000808F500020
:1031B000B7FE3A004200200069C8BF008080FB00D3
:1031C000400220000088B900808144006610B900E8
:1031D0000080E800EF814100A2DE2000E0007900DD
:1031E000030078000100010003FF370069C8BF0039
:1031F0000080FB000880B90064004000E0807C0093
:103200000001EB00706F8000808F5000EAFF3200F9
:1032100069C8BF000080FB00480220000880B90098
:1032200000804400ED004000F00DEC002200200082
:103230008BF707000004E000B5FF3A0069C8BF0043
:103240000080FB000880B90064004000E0807C0042
:1032500012002000A06F8000808F5000D6FF320047
:1032600069C8BF000080FB00480220000880B90048
:1032700000804400ED004000F60DEC00220020002C
:1032800077F707000004E000ACFF3A0069C8BF0010
:103290000080FB000880B90064004000E0807C00F2
:1032A00022002000D06F8000808F5000C2FF3200CB
:1032B00069C8BF000080FB00480220000880B900F8
:1032C00000804400ED004000FC0DEC0022002000D6
:1032D00063F707000004E000A3FF3A0069C8BF00DD
:1032E0000080FB000880B90064004000E0807C00A2
:1032F0003200200000708000808F5000AEFF32004E
:1033000069C8BF000080FB00480220000880B900A7
:1033100000804400ED004000020EEC00220020007E
:103320004FF707000004E00059FE3A0099FF37000C
:10333000080178000201E80023C2BF000008A300D2
:10334000FDFF32000100FB00201188009240780050
:103350000104E00080FE32000201E800F6FF3700C1
:103360000904E8008000EB000000FB0080804000C2
:10337000584078000004E000BDFE32000000FB0071
:1033800080804000584078000004E000F6FF3A00DA
:10339000B7FE37002800FA00889FBE00106E80003C
:1033A000F805070082844700801F7800811F78009D
:1033B00000FF2800801F780009007800EDF6070064
:1033C0001FD89700E68757000004E00017003A0076
:1033D000F2FD2F00028447008000EB00811F78007F
:1033E00020F42800801F780000FD2F000F0040000F
:1033F000E0F60700E6050700E48757000104E00057
:1034000006003200090178000201E800ED0507001E
:10341000FEFF3200CA050700FBFF3A000000EB0088
:103420004F04BE000080FA00000006008000EB00A0
:10343000F2FD2F00028447000000FB008080400066
:10344000584078000004E000E4FF32000000FB0078
:1034500080804000584078000004E000F6FF3A0009
:10346000DEFF37002800FA00889FBE00F06D800064
:10347000C405070082844700801F7800811F780000
:10348000D0FF2800801F780009007800B9F60700F7
:103490001FD89700E68757000004E00017003A00A5
:1034A000F2FD2F00028447008000EB00811F7800AE
:1034B00020F42800801F780000FD2F000F0040003E
:1034C000ACF60700B2050700E48757000104E000EE
:1034D00006003200090178000201E800B905070082
:1034E000FEFF320096050700FBFF3A000000EB00EC
:1034F0004F04BE000080FA00000006008000EB00D0
:10350000F2FD2F00028447000000FB008080400095
:10351000584078000004E000E4FF32000000FB00A7
:1035200080804000584078000004E000F6FF3A0038
:10353000DEFF37002800FA00889FBE00006E800082
:103540009005070082844700801F7800811F780063
:10355000A0002900801F78000900780085F6070088
:103560001FD89700E68757000004E00017003A00D4
:10357000F2FD2F00028447008000EB00811F7800DD
:1035800020F42800801F780000FD2F000F0040006D
:1035900078F607007E050700E48757000104E00085
:1035A00006003200090178000201E80085050700E5
:1035B000FEFF320062050700FBFF3A000000EB004F
:1035C0004F04BE000080FA00000006008000EB00FF
:1035D000F2FD2F00028447000000FB0080804000C5
:1035E000584078000004E000E4FF32000000FB00D7
:1035F00080804000584078000004E000F6FF3A0068
:10360000DEFF37002800FA00889FBE00206E800091
:103610005C05070082844700801F7800811F7800C6
:1036200070012900801F78000900780051F607001A
:103630001FD89700E68757000004E00017003A0003
:10364000F2FD2F00028447008000EB00811F78000C
:1036500020F42800801F780000FD2F000F0040009C
:1036600044F607004A050700E48757000104E0001C
:1036700006003200090178000201E8005105070048
:10368000FEFF32002E050700FBFF3A000000EB00B2
:103690004F04BE000080FA00000006008000EB002E
:1036A000F2FD2F00028447000000FB0080804000F4
:1036B000584078000004E000E4FF32000000FB0006
:1036C00080804000584078000004E000F6FF3A0097
:1036D000DEFF37002800FA00889FBE000004780053
:1036E000306E800001418000E2FD2F00828447009F
:1036F000801F7800811F780030FE2800801F78002E
:10370000090078001BF607003200200088007800CE
:103710007C80570063F607000040EB00F0E79F0055
:103720001FD89700E68757000004E0001C003A000D
:10373000F1FD2F00018447008000EB00811F78001D
:1037400020F42800801F780000FD2F000F004000AB
:1037500008F60700AFD09700014C78003FD19700E2
:1037600012449800D6040700C0EF9F0099407800EB
:10377000E48757000104E0000600320009017800E8
:103780000201E8000F050700FEFF3200EC0407000D
:10379000FBFF3A004F04BE000080FA000000060064
:1037A000F2FD2F00028447008000EB000000FB00C8
:1037B00080804000584078000004E000DFFF3200C5
:1037C0000000FB0080804000584078000004E000CA
:1037D000F6FF3A00D9FF37002800FA00889FBE00A4
:1037E00080007800E0FD2F00808447002210240034
:1037F00033B42400B70407007E80570029F6070081
:10380000D8E79F007FD897000004E00018003A0036
:10381000F1FD2F00018447008000EB00811F78003C
:1038200020F42800801F780000FD2F000F004000CA
:10383000D0F5070081040700C0E79F009940780099
:10384000E48757000104E000060032000901780017
:103850000201E800DE040700FEFF3200BD0407009D
:10386000FBFF3A004F04BE000080FA000000060093
:10387000F1FD2F00018447008000EB000000FB00F9
:1038800080804000584078000004E000E3FF3200F0
:103890000000FB0080804000584078000004E000F9
:1038A000F6FF3A00DDFF37002800FA00889FBE00CF
:1038B00080007800E0FD2F008084470022E0240093
:1038C00013B42400830407007E805700F5F5070039
:1038D000D8E79F00C1040700E2862000624078001C
:1038E0000080FB00801F780041022900811F7800C2
:1038F0007F8057009FF507003FD89700E487570067
:103900000004E00018003A00F0FD2F00008447009A
:103910008000EB00811F780020F42800801F7800D1
:1039200000FD2F000F00400092F507004304070040
:1039300080EF9F0099407800E48757000104E00081
:1039400006003200090178000201E800A004070027
:10395000FEFF32007F040700FBFF3A004F04BE0069
:103960000080FA0000000600F1FD2F0001844700EE
:103970008000EB000000FB00808040005840780091
:103980000004E000E3FF32000000FB008080400004
:10399000584078000004E000F6FF3A00DDFF3700F1
:1039A0002800FA00889FBE008A9FBE006E040700B0
:1039B000660040008A8620008A0478000A004000E1
:1039C0000048EB002104070030C5B30080CF500051
:1039D0005C00320073040700880478000880B90096
:1039E0008A057800000045000048900032C4B3000A
:1039F000824F50000E0132001404070010C4B300BF
:103A000080CF5000E200320036040700660040001C
:103A100042C0B30002707D0062040700490220002A
:103A20000980B9000001450003FD2F008F8141008E
:103A3000EA85410020E0240011B42400808DBE00FE
:103A40000044EB00E8DF9F00E80041003200200066
:103A50006E80410093F5070098E79F00510407002E
:103A60000980B9006600400060407D000080FB00D6
:103A7000801F780040022900801F7800D1FD2F00B0
:103A8000018047003BF507007FD09700E48757008F
:103A90000004E0001D003A00B3FD2F00038447003E
:103AA0008000EB00811F780023F42800831F78003A
:103AB000C0FC2F000F0040002EF507006FC89700D4
:103AC000004C7800FFC8970011449800FC030700E1
:103AD000C0E79F009B407800E48757000104E000A6
:103AE000060032000B0178000201E80038040700EC
:103AF000FEFF320017040700FBFF3A004F05BE002F
:103B00004F04BE000080FA0000000600B1FD2F0047
:103B1000018447008000EB000000FB008080400033
:103B2000584078000004E000DEFF32000000FB0097
:103B300080804000584078000004E000F6FF3A0022
:103B4000D8FF370069C8BF000080FB000880B900BB
:103B500000004500E90040002C0EEC00220020008F
:103B60003FF507000004E0000F003A0069C8BF00FD
:103B70000080FB000880B90064004000E0007D0088
:103B80000001EB0080718000808F5000D200320075
:103B900069C8BF000080FB000880B90066004000D3
:103BA00022C0B30002F07C0069C8BF000080FB00A7
:103BB000480220000880B9008986200000004500E6
:103BC000E9004000320EEC002200200024F507003E
:103BD0000004E0000F003A0069C8BF000080FB004D
:103BE0000880B90064004000E0807C0012002000E2
:103BF000B0718000808F5000B700320069C8BF00EC
:103C00000080FB000880B9006600400022C0B300BD
:103C100002F07C0069C8BF000080FB004802200061
:103C20000880B9008986200000004500E9004000B6
:103C3000380EEC002200200009F507000004E00027
:103C40000F003A0069C8BF000080FB000880B9007F
:103C500064004000E0807C0022002000E0718000D1
:103C6000808F50009C00320069C8BF000080FB00BC
:103C70000880B9006600400022C0B30002F07C005A
:103C800069C8BF000080FB00480220000880B9001E
:103C90008986200000004500E90040003E0EEC004F
:103CA00022002000EEF407000004E0000F003A00BC
:103CB00069C8BF000080FB000880B90064004000B4
:103CC000E0807C003200200010728000808F500065
:103CD0008100320069C8BF000080FB000880B90085
:103CE0006600400022C0B30002F07C0069C8BF003B
:103CF0000080FB00480220000880B900898620006F
:103D000000004500E9004000440EEC0022002000C5
:103D1000D3F407000004E0000E003A0069C8BF00B9
:103D20000080FB000880B90064004000E0807C0057
:103D300040728000808F50006600320069C8BF006A
:103D40000080FB000880B9006600400022C0B3007C
:103D500002F07C0069C8BF000080FB004202200026
:103D60000280B9006600400060407D00E24F5000D4
:103D700029FF320069C8BF000080FB000280B90043
:103D80006600400042C0B30002707D0022FF370091
:103D900069C8BF000080FB000880B9000000450032
:103DA00010489000824F50000800320069C8BF00E0
:103DB0000080FB00420220000280B9006600400043
:103DC00042C0B30002707D0013FF370069C8BF0016
:103DD0000080FB000880B90000004500A04890006A
:103DE000B0C4B30080CF5000F0FF3A0069C8BF00F4
:103DF0000080FB000880B90000004500EB00400097
:103E000032002000B084200095F407008000780084
:103E1000804178000004E0004B003A0010C0B3007D
:103E200047E8B7000100780046E8B700FAFE37001F
:103E300069C8BF000080FB000880B9000000450091
:103E4000E9004000260EEC002200200084F4070068
:103E5000000178000004E0000E003A0069C8BF00CD
:103E60000080FB000980B90064004000E0807D0014
:103E700050718000808F50008000320069C8BF0000
:103E80000080FB000980B9006600400022C0B3003A
:103E900002F07D0069C8BF000080FB0042022000E4
:103EA0000280B9006600400060407D00E24F500093
:103EB000D9FE320069C8BF000080FB000280B90053
:103EC000660040008386200042C0B30002F0790003
:103ED000D1FE37004200200069C8BF000080FB000F
:103EE000480220000880B900660040000A00400037
:103EF0000048EB0069C8BF000080FB000880B900E3
:103F0000800145006610B9000080E800EB814100A7
:103F1000C2E22000E0007900030078000100010007
:103F2000804178000004E0000D003A0069C8BF003D
:103F30000080FB000880B9006600400032C0B3007A
:103F400002707D00B4FE370069C8BF000080FB002E
:103F50000880B9006600400092C0B30002707D0086
:103F6000E1CF5100ACFE3A0069C8BF008080FB0081
:103F7000400220000088B90000014500A0FD2F008C
:103F8000808547002010240031B42400808DBE00BD
:103F90000044EB00E8DF9F00E80041003200200011
:103FA000E3FD2F00038047003EF4070098E79F00E1
:103FB0003FD897000004E00022003A00B0FD2F0037
:103FC000008447008000EB00811F780023F4280064
:103FD000831F7800C0FC2F000F004000E5F30700AE
:103FE0006FC89700004C7800FFC8970011449800F4
:103FF00030C0B300204498000040EB0030449800EB
:1040000080E79F009B407800E48757000104E000B0
:10401000BAFE32000B0178000201E80033C2BF0093
:104020000008A300FDFF32000100FB00A011880082
:10403000924078000104E000B0FE32000201E80086
:10404000F6FF3700B1FD2F00018447008000EB0030
:104050000000FB0080804000584078000004E00031
:10406000D9FF32000000FB008080400058407800FB
:104070000004E000F6FF3A00D3FF370069C8BF0034
:104080000080FB000980B9006600400002F07D005E
:1040900069C8BF000080FB000980B90000804500AE
:1040A0006B004000417180000100010080417800F8
:1040B0000004E000AAFF3A0069C8BF000080FB00CE
:1040C0000980B9006600400032C0B30002F07D00F4
:1040D00051FE37002800FA00889FBE008A9FBE006C
:1040E000D8020700898620000080440070409000BC
:1040F000E24F500066003200C82DA900EB02070015
:10410000640040000001EB0002B07C005302070095
:104110001240980051020700024878004302200034
:1041200002437800A2020700E600420089804000B6
:10413000924098009E020700E700420089804000FC
:104140009240980022002000690207008980400008
:1041500096409800C802070043020700E78040002D
:1041600041020700E88040003F020700E98040006C
:104170003D020700EA8040003B020700EB80400060
:10418000898040009640980066014000FE0F510073
:10419000EDFF3A006968EC0069C8BF00FD4F5000B0
:1041A00035003E009286200012417800E3C1B30042
:1041B000440220002F0207000100320059020700CC
:1041C0005C020700010036000041EB008341E9007A
:1041D0002802070018003A005602070001003600C6
:1041E0000041EB00230207001F003A0051020700C4
:1041F000010036000041EB001E02070012003A00E9
:104200004C020700010036000041EB0019020700D4
:1042100011003A0047020700010036000041EB00A0
:10422000E4C15100E3FF3A004F05BE004F04BE0059
:104230000080FA0000000600C82DA80002007800E7
:1042400069E8B700E4FF3700C82DA8000200780035
:1042500069E8B700EAFF3700C82DA800020078001F
:1042600069E8B700EBFF3700C82DA800020078000E
:1042700069E8B700DDFF37006968EF00928620002B
:1042800012417800E3C1B30044022000C9FF3700A7
:1042900069C8BF000080FB000380B90000804400B3
:1042A0006804400069C8BF000080FB000380B900BB
:1042B0006400400060807C0064055000670050008E
:1042C000FB0F50004C003E000A00E0000D013200E0
:1042D0001841780001CEB30001404100A5C5B300EC
:1042E000854F500044003E008001EB00030278003F
:1042F0000A00E900630060001C0032000202FB00BB
:104300001300200063417C008140410085CF5000B4
:1043100039003E00E10F500014003200E20F50005F
:10432000090032000200FB00000242008301E800A5
:1043300063417C0006CEB30086404100A7C5B300B0
:1043400087CF50002C003E000200FB00000242001C
:104350008301E80063417C0006CEB3008640410043
:10436000A7C5B30087CF500023003E000200FB002A
:10437000000242008302E80085017800850F5500A5
:10438000E100320063417C0006CEB300864041006C
:10439000A7C5B30087CF500017003E000200FB0006
:1043A000000242008501E80063417C0006CEB300B4
:1043B00086404100A7C5B30087CF50000E003E00E5
:1043C0000200FB00000242008581E80063417C009E
:1043D0008640410087CF500007003E000200FB00EE
:1043E00000024200E381420063417C0086404100BC
:1043F00087CF5000DDFF360069C8BF000080FB009A
:104400004A0220000A80B9000080E80060C07C00F9
:10441000E24F500000013200C82DA90069C8BF005A
:104420000080FB00430220000380B90064004000CC
:104430000001EB0002B07C0069C8BF000080FB00F7
:104440000380B9000080E800090040001240980095
:1044500069C8BF000080FB000380B9000080E8004D
:10446000090040000248780002437800918620004D
:10447000914078008180FB00038AB900E600420089
:1044800089804000924098009186200091407800F9
:104490008180FB00038AB900E70042008980400068
:1044A00092409800220020009186200091407800E0
:1044B0008180FB00038AB90084004100E68040004F
:1044C00089804000964098000200E8009186200014
:1044D000914078008180FB00038AB900840040008D
:1044E000E680400089804000964098009186200038
:1044F000914078008180FB00038AB900840040006D
:10450000E780400089804000964098009186200016
:10451000914078008180FB00038AB900840040004C
:10452000E8804000898040009640980091862000F5
:10453000914078008180FB00038AB900840040002C
:10454000E9804000898040009640980091862000D4
:10455000914078008180FB00038AB900840040000C
:10456000EA804000898040009640980091862000B3
:10457000914078008180FB00038AB90084004000EC
:10458000EB80400089804000964098006601400022
:10459000FE0F5100C4FF3A006968EC0069C8BF0013
:1045A000FD4F500051003E009286200012417800DD
:1045B000E3C1B300440220000280FB000480B90084
:1045C00000804400304090000004E000030032000E
:1045D000C82DA8000200780069E8B7000241E80091
:1045E000FD4F5100010036000041EB008341E9001E
:1045F0000280FB000480B90000804400304090003D
:104600000004E00029003A000241E800FD4F51009B
:10461000010036000041EB000280FB000480B9007D
:1046200000804400304090000004E00023003A0085
:104630000241E800FD4F5100010036000041EB004F
:104640000280FB000480B9000080440030409000EC
:104650000004E0001D003A000241E800FD4F510057
:10466000010036000041EB000280FB000480B9002D
:1046700000804400304090000004E00017003A0041
:104680000241E800FD4F5100010036000041EB00FF
:10469000E4C15100C8FF3A004F05BE004F04BE0000
:1046A0000080FA0000000600E3FE3700C82DA800D5
:1046B0000200780069E8B700D3FF3700C82DA800D2
:1046C0000200780069E8B700D9FF3700C82DA800BC
:1046D0000200780069E8B700DFFF3700C82DA800A6
:1046E0000200780069E8B700E5FF37006968EF006D
:1046F0009286200012417800E3C1B30044022000FA
:10470000ADFF37000A027800841F780020F42800EB
:10471000801F780061FD2F000180470015F207001F
:104720008A004400E48757004FD89700914F50000B
:10473000820032000041EB000204E0002EFF320054
:1047400069C8BF000080FB00420220000280B9005F
:104750000080E80060C07C00E24F50008C00320016
:1047600069C8BF000080FB000280B9000080E8003B
:104770008286200060407900E14F500026FF3A0019
:104780002AF90700C82DA90069C8BF000080FB00F6
:10479000430220000380B900640040000001EB00E8
:1047A00002B07C0069C8BF000080FB000380B90034
:1047B0000080E800090040001240980069C8BF006E
:1047C0000080FB000380B9000080E8000900400081
:1047D00002487800024378009186200091407800DA
:1047E0008180FB00038AB900E60042008980400016
:1047F0009240980091862000914078008180FB00D3
:10480000038AB900E7004200898040009240980086
:104810002200200024FF370069C8BF000080FB0091
:104820000A80B9006600400012C0B30002F07C00AC
:1048300069C8BF000080FB000A80B9000081440005
:1048400003FD2F008F814100EA85410020E0240014
:1048500011B42400808DBE000044EB00E8DF9F000F
:10486000E8004100320020006E8041000DF2070098
:1048700098E79F0069C8BF000080FB000A80B9006C
:104880006600400060C07C000080FB00801F780054
:1048900040022900801F7800D1FD2F0001804700D1
:1048A000B4F107007FD09700E48757000004E000D0
:1048B00029003A00B3FD2F00038447008000EB007D
:1048C000811F780023F42800831F7800C0FC2F008C
:1048D0000F004000A7F107006FC89700004C780058
:1048E000FFC897001144980030C0B30020449800DE
:1048F0000040EB0030449800C0E79F009B407800E8
:10490000E48757000104E000C3FE32000B01780089
:104910000201E80033C2BF000008A300FDFF32001F
:104920000100FB00A0118800924078000104E00023
:10493000B9FE32000201E800F6FF37009140900016
:1049400012C0B3005FD89700814F50007AFF320049
:104950000041EB0078FF3700B1FD2F0001844700D4
:104960008000EB000000FB00808040005840780091
:104970000004E000D2FF32000000FB008080400015
:10498000584078000004E000F6FF3A00CCFF370002
:1049900003FC0700C82DA90069C8BF000080FB0008
:1049A000430220000380B900640040000001EB00D6
:1049B00002B07C0069C8BF000080FB000380B90022
:1049C0000080E800090040001240980069C8BF005C
:1049D0000080FB000380B9000080E800090040006F
:1049E00002487800024378009186200091407800C8
:1049F0008180FB00038AB900E60042008980400004
:104A00009240980091862000914078008180FB00C0
:104A1000038AB900E7004200898040009240980074
:104A200022002000A0FE37000041780000CDB30036
:104A300000404100E94F500000000600EFC8970019
:104A4000014C78001C00070000000600250007004C
:104A50000000450080489000000006008D0007001F
:104A60000900400000000600898040009640980040
:104A7000230037000280FB000480B900008044005E
:104A8000304090000004E000000006007E000700B7
:104A90008301E80063417C0007CEB30087404100FA
:104AA000A6C5B30086CF50000000060086804000F7
:104AB00097409800120037003FC8970010449800B4
:104AC00030C0B300204498000040EB003044980010
:104AD00000000600828CBE000044EB00E8DF9F006F
:104AE000320005002F0007000880B9000000060012
:104AF0002F00070084004100E6804000000006000F
:104B00002B00070084004000000006000280FB002C
:104B10000480B90000004300304090000004E00031
:104B200000000600C82DA8000200780069E8B70060
:104B3000000006000241E800FD4F510000000600A1
:104B40000100FB0020118800924078000104E00081
:104B5000000006000100FB00A011880092407800D0
:104B60000104E000000006000E00070048022000DB
:104B70000880B90000000600DAFF0700008044004A
:104B800000000600316E8000E2FD2F0000000600EC
:104B90006FC99700024C7800C7FF07009940780062
:104BA0000000060069C8BF000080FB00000006008E
:104BB00091862000914078008180FB00038AB90033
:104BC0000000060023C2BF000008A300000006008A
:104BD00033C2BF000008A30000000600F1FF070079
:104BE000420220000280B9000000060090407800D8
:104BF000E1F79F0090409000F1F79F00A0409000E7
:104C000081FF9F003040900090FF9F000040EB002C
:104C1000A0FF9F0000000600800078000001EB006C
:104C2000F0702200808F5000000006000001780024
:104C3000EA0050008001EB00600E2000808F5000E1
:104C400000000600D7FF0700430220000380B900E0
:104C500000000600150007000000410000000600EB
:104C60000C00070006004000000006000C000700D2
:104C700097409800000006000200E800A0FF07002F
:104C8000E6804000000006000200FB000002420037
:104C900000000600050007000080E8000000060094
:104CA00093FF07008680400000000600BDFF07005C
:104CB0000380B900000006009A03070042C7BF0046
:104CC0000058A300FDFF3200000006000000EB00CA
:104CD00020048800300488004004880050048800C4
:104CE00060048800000006009A0307008000EB00C3
:104CF000B1168800000C2000C0168800E11688005C
:104D000050052000F016880011178800970307004F
:104D1000000006009A030700000006009E0307003B
:104D2000C00A200040118800A4030700000006000C
:104D30003062A8003002A90030C2BF0091CFB3009A
:104D4000AB030700C00A2000C0118800AD030700B4
:104D5000000006002023A9002043A8002063A9002A
:104D600003CEB300034078002063B70021C3BF0027
:104D7000C2CFB30002406000AF03070002406000F2
:104D8000B803070003406000C00307008000EB0089
:104D900031198800411988007000200080198800AE
:104DA000811B8800C203070000000600C70307003C
:104DB000C1CFB30001406000CE0307000000060031
:104DC000D7030700C1CFB30001406000DE03070036
:104DD00000000600F0030700C1CFB30001406000EF
:104DE000C0E1B700F0F32100200E88000000EB00C6
:104DF000B00E8800C00E8800D00E8800E00E88003B
:104E0000F003070001C4B30001407000CCE1B7001B
:104E1000CDC1BF00F043B20001407000F9030700AC
:104E2000000006008460A900A5C0BF00F1C8B3005F
:104E30000C0407000000060084E0A900A7C0BF0022
:104E4000F1C8B30016040700000006008E0F07002B
:104E5000F20D0700FE0D07009860A8000C04A800E2
:104E60000C24A800000006001B0407000000060038
:104E70008040780023040700FEFF3A002404070066
:104E80000000060025040700FEFF320040138000EA
:104E90000080FB000000060023040700FD4F5000C7
:104EA00003003E00A1D6200027040700FEFF3600C5
:104EB000A86DEF00E9090700306B8800416B88009E
:104EC00000000600889FBE002804070026CA2000B4
:104ED0004884200005822000034278001905200044
:104EE000030307000300E80004F07B0004707B006C
:104EF00066014000010307008001E800FC02070092
:104F00008081E80084F17B0084717B0068014000AF
:104F1000880041003004070084717B006901400073
:104F2000880041003004070084717B006A01400062
:104F3000880041003004070084717B006B01400051
:104F4000880041003004070084717B006C01400040
:104F5000880041003004070084717B006D0140002F
:104F60008800410030040700DDFF3A0032040700EA
:104F70004204070046040700FEFF3A005A040700F7
:104F8000FBFF3A005D0407004F04BE00000006006E
:104F90007304070054090700DA030700FEFF3A0014
:104FA0006000200040138800DC030700FEFF320091
:104FB0006D0407004C093700690407004A0907001F
:104FC000D0030700FEFF3A00400020004013880095
:104FD000D2030700FEFF32006304070042093700D6
:104FE000881F78005E0407003F090700C50307001B
:104FF000FEFF3A005000200040138800C70307005E
:10500000FEFF320040138000BE030700FEFF3A009F
:105010006822EF00C1030700FEFF320055040700BD
:10502000310907000880FB004F04780000000600EB
:10503000881F780052040700200020002A0907007A
:10504000E7FF07000008A300020032004E0407003B
:10505000F9FF36004F04780000000600881F780032
:1050600047040700200020001F090700DCFF07009D
:105070000018A30002003A0043040700F9FF3600BD
:105080004F04780000000600889FBE008A9FBE0083
:1050900080047800810578003104070012090700B8
:1050A00098030700FEFF3A003000200040138800FC
:1050B0009A030700FEFF320040138000C848DE005C
:1050C00090030700FEFF3A009103070093030700D7
:1050D000FEFF3200401380008940780089030700FA
:1050E000FEFF3A008A0307008C030700FEFF320030
:1050F0004013800083030700FEFF3A006822EF00A0
:1051000086030700FEFF32001A040700F6080700B6
:105110004845DD0020002000F308070010040700C8
:10512000F108070077030700FEFF3A003000200077
:105130004013880079030700FEFF3200401380000F
:105140000901E800C810DE006E030700FEFF3A0008
:105150006F03070071030700FEFF32004013800059
:105160008240780067030700FEFF3A0068030700EB
:105170006A030700FEFF320040138000610307004E
:10518000FEFF3A006822EF0064030700FEFF3200D2
:10519000F8030700D40807000884FB00880D4500C9
:1051A0004F05BE004F04BE0000000600889FBE00F1
:1051B0008A1F78008004780001057800E803070062
:1051C000C90807004F030700FEFF3A0060002000F7
:1051D0004013880051030700FEFF3200E20307007E
:1051E000C1080700E603070020002000BE080700F2
:1051F0007BFF07000018A30002003A00E20307004B
:10520000F9FF3600D6030700B70807003D03070083
:10521000FEFF3A0020002000401388003F030700F3
:10522000FEFF320040138000C848DE00350307004F
:10523000FEFF3A003603070038030700FEFF320086
:1052400040138000894078002E030700FEFF3A00DB
:105250002F03070031030700FEFF320040138000D8
:10526000C850DE0027030700FEFF3A0028030700AE
:105270002A030700FEFF3200BB0307009A0807005D
:10528000BF030700200020009708070054FF070015
:105290000008A30002003200BB030700F9FF36003C
:1052A000AF0307009008070016030700FEFF3A004F
:1052B000600020004013880018030700FEFF320042
:1052C000A903070088080700AD030700200020009D
:1052D0008508070042FF07000018A30002003A00FB
:1052E000A9030700F9FF36009D0307007E080700A9
:1052F00004030700FEFF3A0020002000401388004E
:1053000006030700FEFF3200401380000901E80099
:10531000C810DE00FB020700FEFF3A00FC02070097
:10532000FE020700FEFF320040138000824078003A
:10533000F4020700FEFF3A00F5020700F70207003B
:10534000FEFF3200401380008A407800ED02070023
:10535000FEFF3A00EE020700F0020700FEFF3200F7
:105360008103070060080700850307002000200074
:105370005D0807001AFF07000008A30002003200C2
:1053800081030700F9FF3600750307005608070080
:10539000DC020700FEFF3A004000200040138800B6
:1053A000DE020700FEFF32006F0307004E08070011
:1053B0004F0578004F04BE0000000600810278000F
:1053C0008400780015027800820F52000200390034
:1053D000830F520002003600810A780073FF070035
:1053E000000006008009290021F507003006200092
:1053F000306E8800316E8000000120006BFF0700D6
:10540000401F2000206E8800216E800020012000B7
:1054100066FF070040062000006E8800016E8000D5
:105420004001200061FF0700000F2000F06D8800A0
:10543000F16D8000600120005CFF0700800C2000FF
:10544000106E8800116E80008001200057FF370029
:105450000200FA0001AA2A00000F200053FF0700F3
:1054600011AA2A00200F200050FF070021AA2A00BD
:10547000400F20004DFF070031AA2A00600F2000D6
:105480004AFF070041AA2A00800F200047FF0700BB
:1054900051AA2A00A00F200044FF070061AA2A0099
:1054A000C00F200041FF070071AA2A00E00F200072
:1054B0003EFF07008F80E900000F2000F2FE07008A
:1054C00000AA2A003303070076003A008F80E90023
:1054D000200F2000ECFE070010AA2A002D03070071
:1054E00070003A008F80E900400F2000E6FE0700C0
:1054F00020AA2A002A0307006A003A008F80E900E8
:10550000600F2000E0FE070030AA2A0021030700F8
:1055100064003A008F80E900800F2000DAFE070067
:1055200040AA2A001E0307005E003A008F80E900AF
:10553000A00F2000D4FE070050AA2A001503070080
:1055400058003A008F80E900C00F2000CEFE07000F
:1055500060AA2A001203070052003A008F80E90077
:10556000E00F2000C8FE070070AA2A000C03070005
:105570004C003A0001BB2B00000F20000BFF07007E
:1055800011BB2B00200F200008FF070021BB2B00C0
:10559000400F200005FF070031BB2B00600F2000EB
:1055A00002FF070041BB2B00800F2000FFFE070019
:1055B00051BB2B00A00F2000FCFE070061BB2B009D
:1055C000C00F2000F9FE070071BB2B00E00F200088
:1055D000F6FE07008F80E900000F2000AAFE0700FA
:1055E00000BB2B00EB0207002E003A008F80E90081
:1055F000200F2000A4FE070010BB2B00E8020700CC
:1056000028003A008F80E900400F20009EFE07002E
:1056100020BB2B00DF02070022003A008F80E90048
:10562000600F200098FE070030BB2B00DC02070053
:105630001C003A008F80E900800F200092FE0700D6
:1056400040BB2B00D302070016003A008F80E90010
:10565000A00F20008CFE070050BB2B00D0020700DB
:1056600010003A008F80E900C00F200086FE07007E
:1056700060BB2B00C70207000A003A008F80E900D8
:10568000E00F200080FE07001100200070BB2B00FF
:10569000C302070003003A00010078000080FA000E
:1056A00000000600000020000080FA000000060054
:1056B000FCFF3700881F780065FF07000000E0004E
:1056C00069003200C80DA800D4C2BF000068A30062
:1056D0004D00320061DC2000000120006AFE07005E
:1056E000316E80000100E0004E00320030062000E4
:1056F000808F50004B003E0048DC2000880078007E
:105700002001200060FE0700A80207004F003E00B5
:1057100001DC2000400120005BFE0700016E8000DC
:10572000E98F500033003600000F2000808F5000BA
:1057300030003E00E1DB20006001200052FE070047
:10574000F16D8000E98F50001F003600000F20002F
:10575000808F50001C003E0028DC2000880078006C
:105760008001200048FE07009002070011003E0063
:10577000206E80000000E00001003A00A06A88006E
:10578000C8CDBF000008A30035003A00480620003D
:10579000C01220004F070700CAE2A800C86A8800AC
:1057A000C01220004B070700CAE2A800C86A8800A0
:1057B000F7FF370081252000116E8800800120004E
:1057C0007AFE0700EAFF370041062000F16D8800ED
:1057D0006001200075FE070028DC200088007800AA
:1057E0008001200028FE070070020700E0FF36005D
:1057F000F0FF370061042000016E880040012000A6
:105800006AFE0700CBFF3700F6FE070061DC2000D0
:10581000000120001CFE0700316E80000100E00046
:10582000B2FF3A0031062000316E880000012000EE
:105830005EFE070048DC2000880078002001200080
:1058400011FE070059020700B1FF3600411F20007A
:10585000216E88002001200054FE0700ACFF3700B5
:105860004F04780000000600C80DA900D4C2BF0094
:105870000068A30097FF3A00E3FF3700889FBE004F
:10588000A800070042C7BF000058A300FDFF320078
:105890008420EF008620EF008820EF008A20EF00B0
:1058A0008C20EF00AB000700D622EF00000C200098
:1058B000C0168800DC22EF0050052000F01688009A
:1058C000E222EF00A900070033010700C8CFB300B0
:1058D00008406000C0E1B700F0F32100200E88000E
:1058E000D621EF00D821EF00DA21EF00DC21EF0014
:1058F000340107000064A000CCE1B700CDC1BF00B7
:10590000F043B2000064A0003E010700DE0C070077
:10591000420B07004E0B07009860A8000C04A8007B
:105920000C24A8009C000700C20A20004211880035
:10593000A20007003062A8003002A90030C2BF00F8
:10594000AB000700C2118800AE0007002023A900A9
:105950002043A8002063A90002CEB30002407800D3
:105960002063B70021C3BF0008406000B2000700F9
:1059700008406000BB00070002406000C300070051
:105980002623EF002823EF007000200080198800F4
:105990007023EF00C6000700CC000700084060003D
:1059A000D4000700DE00070008406000E6000700A2
:1059B0008460A900A5C0BF002A01070084E0A900F7
:1059C000A7C0BF00360107003AFF070067010700C4
:1059D00028CA200046842000058220000342780067
:1059E000190520004A0007000300E80004F07B00CE
:1059F00004707C0066014000480007008001E80058
:105A0000430007008081E80084F17B0084717C0002
:105A100068014000860041006F01070084717C002E
:105A200069014000860041006F01070084717C001D
:105A30006A014000860041006F01070084717C000C
:105A40006B014000860041006F01070084717C00FB
:105A50006C014000860041006F01070084717C00EA
:105A60006D014000860041006F010700DDFF3A0034
:105A7000710107008101070085010700FEFF3A0060
:105A800099010700FBFF3A009C010700260107006F
:105A9000A1D62000FD4F500002003E002A01070061
:105AA000FEFF3600A86DEF00EC060700306B8800A3
:105AB000416B88003200070007010700DC42A900A3
:105AC0004006200083060700DC42A800DC62A90033
:105AD000B0CDBF00E24F5000FDFF36004F04BE00C6
:105AE0000000060065FF0700450A070010000500DA
:105AF00084F17B0084717B00668141008800410055
:105B00008048EB00850041008048EB000000060063
:105B100084F17B0084717C00668141008600410035
:105B2000F7FF370060022000303A880044C7BF000A
:105B3000F043B20044E7B70044C7BF0001CEB30052
:105B40000140600044E7B7004827EF0040A7A900E4
:105B500000000600F0112A003016880000E0210045
:105B600050168800D2A2EF00000006008008200036
:105B70002017880040002000401788000000060021
:105B800060A0A90060C0A90068A0A90068C0A90021
:105B90009660A900000006002062A8002002A9006B
:105BA00020C2BF0091CFB3000140600020E2B700E7
:105BB00020A2A9002162A8000000060023A2A900DB
:105BC00023E2A90022C2BF00F043B20022E2B700E4
:105BD00021E2A8002342A8009C20A8009580A900EB
:105BE0009560A8008580A9008560A90000000600D6
:105BF0000140600030E2B70030A2A9003162A80085
:105C00000000060033A2A90033E2A90032C2BF009F
:105C1000F043B20032E2B70031E2A8003342A800FC
:105C20009C40A80097E0A90097C0A80087E0A900C1
:105C300087C0A9000000060021E3B7002143A800A7
:105C40002183A9002223A90022C3BF0031CCB300C5
:105C5000014060000034A00022E3B70023C3BF006E
:105C60000000060023E3B7002343A8002203A90095
:105C700023C3BF007F40600023E3B70060C0B300D0
:105C800024E3B70025C3BF00000006000004A00005
:105C900025E3B70025E3A90032C3BF0081CFB300DD
:105CA000014060000014A00032E3B70000000600CD
:105CB00080FF2F00601988006CA3EF0085A0A90069
:105CC00095A0A90021E3A80000000600D000200054
:105CD000701C880000302000A01C88008CC3BF000E
:105CE000F1CCB300014060008CE3B7008CC3BF006F
:105CF000000006008CE3B7008DA3A9008DC3A900A6
:105D0000F0022000B01C8800007A2000801C88006F
:105D10008DE3A80085C0A80095C0A800000006007B
:105D20006382A9006362A9006342A9006322A900FB
:105D30006302A80062C2A90062A2A80062E2A900F0
:105D400062C2BF00000006000014A00062E2B700BB
:105D500062C2BF0031CEB3000140600062E2B70012
:105D600065E2A90065A2A9006422A90061A2A800B9
:105D700060C2A90061E2A8008820A9009820A900BB
:105D8000B4C0BF00F1C8B300014060000064A000CF
:105D9000B4E0B70000000600C1E1A900C1A1A8005D
:105DA000C0C1BF006F406000C0E1B700C0C1BF000C
:105DB00031CFB30001406000C0E1B700C0C1BF00F7
:105DC00000000600C901A900C921A900C941A90014
:105DD000C961A900C801A900C821A900C841A9003A
:105DE000C861A900C881A800C8A1A900C8C1A800AD
:105DF000C8E1A900CA41A900CCC1BF00F043B2006C
:105E000000000600CDE1B700CCC1BF0001CCB3005B
:105E100001406000CCE1B700CDC1BF00014060008F
:105E2000CDE1B700CE01A900CE21A900CE41A90045
:105E3000CE61A900CE81A900CEA1A900CEC1A90042
:105E4000CEE1A9009BE0A8008BE0A9009C00A8007F
:105E50008C00A900C1E1A8009B20A8008B20A9000C
:105E600000000600014060000064A000A5E0B7004B
:105E70009460A80005E1A90005A1A90004C1A9003A
:105E800004A1A9000481A8000441A9000421A900DB
:105E9000803821001008880005E1A80000000600F5
:105EA000014060000045B300A7E0B70094E0A900FE
:105EB00011E1A90011A1A90010C1A90010A1A90018
:105EC0001081A8001021A900401F20006008880050
:105ED00011E1A900000006008200A8008220A800AD
:105EE0008240A8008260A8008280A8009400A800D8
:105EF0009680A90097A0A8009AA0A9009AC0A9001E
:105F00000000060060C2BF000018A30000000600E9
:105F10000180FB00401388000000060060C2BF0043
:105F20000008A30000000600622DEF00602DEF00C6
:105F30005C2DEF00F00F2000F06A8800A86DEF00E4
:105F4000A8CDBF0000000600A8CDBF000080FB0068
:105F500000004000F26A800002B07800A86DEC00FA
:105F6000A8CDBF00FD4F500000000600B36DEF004C
:105F7000B26DEF00B16DEF00B06DEF00B42DEF002A
:105F8000AE2DEF00AC2DEF00AA2DEF002003200076
:105F9000B06A8800C82DEF00CA2DEF001A68EF0024
:105FA000BC2DEF00BA2DEF00B82DEF00B62DEF009D
:105FB0004C2DEF004A2DEF00482DEF00462DEF004D
:105FC000442DEF006868EF006968EF008001EB0086
:105FD00037CF200000000600C9FE0700E3014000A3
:105FE00084F17B0000000600C5FE0700E4014000CC
:105FF00084F17B0000000600C1FE0700E5014000BF
:1060000084F17B0000000600BDFE0700E6014000B1
:1060100084F17B0000000600B9FE0700E7014000A4
:1060200084F17B0000000600B5FE0700E801400097
:10603000898F5100000006004868EF004668EF00B5
:106040004768EF004428EF004968EF002468EF003C
:106050002268EF002368EF002028EF002568EF009A
:106060000003EB00888620004702200006427800EB
:10607000A2862000C3862000000006008002EB00FC
:1060800007B0B90000004400E7004000000006002F
:106090004900070001007800470007004B00070097
:1060A0008080E80049000700E30040004700070047
:1060B000E400400045000700E50040004300070001
:1060C000E600400041000700E70040003F000700F5
:1060D000E80040003D000700E9004000EA8242007D
:1060E000FE8F5200000006000603E8004302B000E5
:1060F0004202B000FE0F530000000600DC6DEF000E
:10610000D46DEF00CC6DEF00DD6DEF00D56DEF00CD
:10611000CD6DEF00DE6DEF00D66DEF00CE6DEF00C0
:10612000DF6DEF00D76DEF00CF6DEF00E06DEF009A
:10613000D86DEF00D06DEF00E16DEF00D96DEF008D
:10614000D16DEF00E26DEF00DA6DEF00D26DEF0080
:10615000E36DEF00DB6DEF00D36DEF000000060094
:10616000E842A9002000050040138000E842A80092
:106170002000050048138000E842A8002000050028
:10618000B42DEF00883E0500A06D8000880F500000
:1061900000000600DFB89700808F50000000060066
:1061A0005FB99700800F510000000600F0702200D8
:1061B000980F1000000006000049EB001441980001
:1061C0008009EB008058EB00000006000049EB005E
:1061D000144198008009EB008048EB0000000600A5
:1061E0003600F800809FBE00829FBE00849FBE00E4
:1061F000869FBE008460A900B42DEC00AC2DEC009D
:10620000580DE20003003400582DED00580DE20057
:106210005E003200560DE2005F003400562DED00A6
:10622000560DE2001F003200B36DEC00B3CDBF008D
:10623000E94F500015003600B36DEF00B26DEC0071
:10624000B2CDBF00E94F500010003600B26DEF0034
:10625000AA2DEC00C86DA800B16DEC00B1CDBF0057
:10626000E94F500009003600B16DEF00C88DA8005D
:10627000B06DEC0001DB200091407800B0C3B300AA
:1062800080CF500001003600B06DEF004F03BE001C
:106290004F02BE004F01BE004F00BE003600F900A5
:1062A0000040060020032000B06A8800E0C2BF0062
:1062B0000068A3003B003200CAEDA900C9C2BF00BC
:1062C0000058A3003B003A001A08A800C942E200A7
:1062D0003B0035001A28A800D5C2BF000028A30043
:1062E0003B003A001A48A800D5C2BF000038A300FE
:1062F0003B003A001A68A800E6C2BF000038A300BD
:106300003B003A001A88A8001AC8BF00D4EDB700B5
:10631000506E8000D5EDB700DECDBF00D6EDB700E2
:10632000DFCDBF00D7EDB700E0CDBF00D8EDB7009F
:10633000E1CDBF00D9EDB700E2CDBF00DAEDB70087
:10634000E3CDBF00DBEDB700CBC2BF004200DE00F3
:10635000610060000004A2004200DD00B12C2000BA
:10636000914078000124A10080C0700001007800F5
:10637000CBE2B7002300200042DD200020032000F4
:1063800001002000160A0700A7FF3700CAE2A90093
:10639000560DE200A1FF3C0020032000B06A8800F7
:1063A000A1FF3700CAEDA800C9C2BF000058A30072
:1063B000C5FF32001A08A900C942E200C5FF3D002E
:1063C0001A28A900D5C2BF000028A300C5FF3200CB
:1063D0001A48A900D5C2BF000038A300C5FF32008B
:1063E0001A68A900E6C2BF000038A300C5FF32004A
:1063F0001A88A9001AC8BF00D4EDB700506E8000FB
:10640000D5EDB700DECDBF00D6EDB700DFCDBF00C4
:10641000D7EDB700E0CDBF00D8EDB700E1CDBF00AC
:10642000D9EDB700E2CDBF00DAEDB700E3CDBF0094
:10643000DBEDB700CBC2BF004200DE0061006000B0
:106440000004A2004200DD00B12C20009140780041
:106450000124A10080C0700001007800CBE2B700E9
:106460002300200042DD2000200320000100200046
:10647000DB0907006CFF370084E0A900004006003C
:106480003600F800809FBE00829FBE00849FBE0041
:10649000869FBE008860A9000AC4BF000008A30050
:1064A000010032000A04A9000AC4BF000018A300BA
:1064B0000600320020C4BF000018A30014003A00F8
:1064C000008020006A0907000A24A90020408000FB
:1064D00031408000EA0F5000E08F58001B0032006E
:1064E000F40F5000E08F580020003200F50F5000EC
:1064F000E08F58000D0032004F03BE004F02BE0077
:106500004F01BE004F00BE003600F90000400600FB
:1065100010C0B30003E8B7002024A90000802000C9
:10652000530907000A24A900E8FF3700370C0700C9
:106530004F03BE004F02BE004F01BE004F00BE0021
:106540003600F90000400600F1FF37000C0C070090
:106550004F03BE004F02BE004F01BE004F00BE0001
:106560003600F90000400600E9FF37001F0C070065
:106570004F03BE004F02BE004F01BE004F00BE00E1
:106580003600F90000400600E1FF3700809FBE00A2
:10659000829FBE00849FBE00869FBE00881F780039
:1065A0008560A9003111800001417800506A8000A7
:1065B00034CF200001707A00516A8000F00420007E
:1065C000808F500009003C004A2DEC00E34F510041
:1065D000090032004F0478004F03BE004F02BE0096
:1065E0004F01BE004F00BE00004006004A2DEF00E4
:1065F000E34F5100F7FF3A000001EB0036CF2000D7
:10660000F304200082427800A7C7B300406A8000EC
:1066100060407A00E24F50003D003200406A800046
:1066200060407B00E34F50008E003200406A8000E3
:1066300005707A00406A8000830F500096003C008D
:10664000482DEC000201E800406A800060407A00BA
:10665000E24F500096003200406A800060407B00AC
:10666000E34F50007F003200406A800005707A00DE
:10667000406A8000830F50009C003400482DEF00DA
:10668000406A800060407A00E24F50009C00320077
:10669000406A800060407B00E34F50007100320090
:1066A000406A800005707A00406A8000830F5000C5
:1066B000A2003400482DEF00406A800060407A005C
:1066C000E24F5000A2003200406A800060407B0030
:1066D000E34F500063003200406A800005707A008A
:1066E000406A8000830F5000A8003400482DEF005E
:1066F0006301410000052000800F5100B5FF32000A
:10670000406A800060407A00E24F5000C3FF3A00C8
:10671000406A80008000EB00830F500001003C00C5
:106720008000E80061407A00FF4F5000BFFF340056
:1067300061407A00874F5000BCFF3C00C82DA80084
:1067400068C8BF000080FB00420220000280B90040
:106750000080E8008686200013C0B30003707B0031
:1067600068C8BF000080FB000280B9000000430041
:10677000334098008002EB008203780005447800E3
:10678000406A800060407A00E24F500021003200F1
:106790008501E80068C8BF000080FB00426A8000F5
:1067A0000780B900008042000000430062417A0087
:1067B00072409800406A800008707A00406A800049
:1067C00008707A00416A8000F0042000808F500039
:1067D00022003C00482DEC0068C8BF000080FB0090
:1067E0000780B90000804200000043007040900024
:1067F000E34F50007A003200FD8F510077003C00DB
:1068000083027800406A800060407A00E24F5000C6
:10681000DFFF3A008002EB001300200068C8BF00D1
:106820000080FB00426A80000780B90000804200BF
:106830000000430062417A0072409800406A800084
:1068400008707A00406A800008707A00416A80000F
:10685000F0042000808F5000DEFF3400482DEF0050
:10686000DDFF3700406A800005707B00406A8000D1
:10687000830F500051003C00482DEC004F0478007D
:106880004F03BE004F02BE004F01BE004F00BE00CE
:106890000040060055FF3700482DEF000201E800D8
:1068A000406A800060407A00E24F50006AFF3A0080
:1068B000406A8000830F50003A003C008000E800EE
:1068C00061407A00FF4F500067FF340061407A005A
:1068D000874F500099FF3400406A800005707A00AD
:1068E000406A8000830F500064FF3C00482DEC009C
:1068F000406A800060407A00E24F500064FF3A0036
:10690000406A8000830F500028003C008000E800AF
:1069100061407A00FF4F500061FF340061407A000F
:10692000874F500085FF3400406A800005707A0070
:10693000406A8000830F50005EFF3C00482DEC0051
:10694000406A800060407A00E24F50005EFF3A00EB
:10695000406A8000830F500016003C008000E80071
:1069600061407A00FF4F50005BFF340061407A00C5
:10697000874F500071FF3400406A800005707A0034
:10698000406A8000830F500058FF3C00482DEC0007
:106990006301410000052000800F510058FF3A00BC
:1069A0000CFF37008000EB00C5FF37008000EB00D4
:1069B000D7FF37008000EB00E9FF3700482DEF00DC
:1069C0004F0478004F03BE004F02BE004F01BE00CF
:1069D0004F00BE000040060004FF37008301E800BE
:1069E00068C8BF000080FB00420220000280B9009E
:1069F0006400400003307B006868EC0068C8BF009A
:106A0000FD4F5000F3FE36006868EF004F04780039
:106A10004F03BE004F02BE004F01BE004F00BE003C
:106A200000400600F1FE3700809FBE00829FBE003E
:106A3000849FBE00869FBE00889FBE0087C0A900BD
:106A4000B111800001417800306A800024CA200022
:106A500001707A00316A8000F0042000808F5000BD
:106A600009003C00462DEC00E34F510009003200C4
:106A70004F04BE004F03BE004F02BE004F01BE00D8
:106A80004F00BE0000400600462DEF00E34F5100CE
:106A9000F7FF3A008001EB0037CF200026CA200024
:106AA000F504200003417800206A800060407A00ED
:106AB000E24F500045003200206A800060407B00B9
:106AC000E34F500094003200206A800002707A0088
:106AD000206A800002F07B00206A8000850F500051
:106AE0009C003C00442DEC008301E800206A8000FB
:106AF00060407A00E24F50009C003200206A800023
:106B000060407B00E34F500083003200206A800029
:106B100002707A00206A800002F07B00206A800008
:106B2000850F5000A3003400442DEF00206A800040
:106B300060407A00E24F5000A3003200206A8000DB
:106B400060407B00E34F500073003200206A8000F9
:106B500002707A00206A800002F07B00206A8000C8
:106B6000850F5000AA003400442DEF00206A8000F9
:106B700060407A00E24F5000AA003200206A800094
:106B800060407B00E34F500063003200206A8000C9
:106B900002707A00206A800002F07B00206A800088
:106BA000850F5000B1003400442DEF00E381410017
:106BB00000052000808F5100ADFF3200206A800068
:106BC00060407A00E24F5000BBFF3A00206A80002C
:106BD0008000EB00850F500001003C008000E800C1
:106BE00061407A00FF4F5000B7FF340061407A00E7
:106BF000A1C7B300814F5000B3FF3C00C82DA800CF
:106C000068C8BF000080FB00430220000380B90079
:106C10000080E8008886200022C0B30002707C005B
:106C200068C8BF000080FB000380B900000044007A
:106C300012C0B300324098008002EB008544780017
:106C4000206A800060407A00E24F50009D003200D0
:106C5000050378008502E80068C8BF000080FB00DB
:106C6000236A8000420220000280B9000000430035
:106C700000004400E3417A0073409800206A8000DD
:106C800009707A00206A800009F07B00216A800088
:106C9000F0042000808F500088003C00442DEC0060
:106CA00068C8BF000080FB00420220000280B900DB
:106CB000000043000000440070409000E34F50008B
:106CC00003003200FD8F5200DDFF34008502E80032
:106CD00068C8BF000080FB000280B900640040006B
:106CE00082862000053079006868EC0068C8BF0023
:106CF000FD4F50005EFF36006868EF004F04BE0095
:106D00004F03BE004F02BE004F01BE004F00BE0049
:106D1000004006005CFF3700206A800002707B00A4
:106D2000206A800002F07B00206A8000850F5000FE
:106D30005A003C00442DEC004F04BE004F03BE003F
:106D40004F02BE004F01BE004F00BE0000400600D3
:106D50004DFF3700442DEF008301E800206A8000DA
:106D600060407A00E24F500064FF3A00206A8000E1
:106D7000850F500043003C008000E80061407A002D
:106D8000FF4F500061FF340061407A00A1C7B3009B
:106D9000814F500099FF3400206A800002707A0011
:106DA000206A800002F07B00206A8000850F50007E
:106DB0005DFF3C00442DEC00206A800060407A00BA
:106DC000E24F50005DFF3A00206A8000850F5000BE
:106DD0002E003C008000E80061407A00FF4F500028
:106DE0005AFF340061407A00A1C7B300814F5000C0
:106DF00082FF3400206A800002707A00206A8000DE
:106E000002F07B00206A8000850F500056FF3C0096
:106E1000442DEC00206A800060407A00E24F500070
:106E200056FF3A00206A8000850F500019003C0090
:106E30008000E80061407A00FF4F500053FF3400AB
:106E400061407A00A1C7B300814F50006BFF34004E
:106E5000206A800002707A00206A800002F07B00C5
:106E6000206A8000850F50004FFF3C00442DEC004D
:106E7000E381410000052000808F51004FFF3A0060
:106E8000FBFE37008000EB00BCFF37008000EB000A
:106E9000D1FF37008000EB00E6FF3700442DEF0004
:106EA0004F04BE004F03BE004F02BE004F01BE00A4
:106EB0004F00BE0000400600F3FE3700442DEF00F7
:106EC00077FF37000003EB001500200062FF37005A
:106ED0003600F800809FBE00829FBE00849FBE00E7
:106EE000869FBE008BE0A900650107002B003200E1
:106EF000500020007C0107006401070027003A00D1
:106F000050002000780107006001070023003A00CC
:106F100050002000740107005C0107001F003A00C8
:106F20005000200070010700580107001B003A00C4
:106F3000500020006C0107005401070017003A00C0
:106F400050002000680107005001070013003A00BC
:106F500050002000640107004C0107000F003A00B8
:106F60005000200060010700480107000B003A00B4
:106F7000500020005C0107004401070007003A00B0
:106F800050002000580107004001070003003A00AC
:106F900041010700A002290035EE07004F03BE00A3
:106FA0004F02BE004F01BE004F00BE003600F90088
:106FB000004006003600F800809FBE00829FBE00A1
:106FC000849FBE00869FBE008C00A9002C01070094
:106FD0002B0032005000200043010700370107005A
:106FE00027003A00500020003F010700330107004E
:106FF00023003A00500020003B0107002F0107004A
:107000001F003A0050002000370107002B01070045
:107010001B003A0050002000330107002701070041
:1070200017003A00500020002F010700230107003D
:1070300013003A00500020002B0107001F01070039
:107040000F003A0050002000270107001B01070035
:107050000B003A0050002000230107001701070031
:1070600007003A00500020001F010700130107002D
:1070700003003A000801070030042900FCED070076
:107080004F03BE004F02BE004F01BE004F00BE00C6
:107090003600F900004006003600F800809FBE0070
:1070A000829FBE00849FBE00869FBE008400A90010
:1070B000A00020000C010700030107002C003A008B
:1070C000A000200008010700FF00070028003A0088
:1070D000A000200004010700FB00070024003A0084
:1070E000A000200000010700F700070020003A0080
:1070F000A0002000FC000700F30007001C003A007D
:10710000A0002000F8000700EF00070018003A0078
:10711000A0002000F4000700EB00070014003A0074
:10712000A0002000F0000700E700070010003A0070
:10713000A0002000EC000700E30007000C003A006C
:10714000A0002000E8000700DF00070008003A0068
:10715000CAE2A80020032000C06A8800CB82A900F0
:1071600011002000007D200030090700CAEDA800B2
:107170004F03BE004F02BE004F01BE004F00BE00D5
:107180003600F900004006003600F800809FBE007F
:10719000829FBE00849FBE00869FBE008680A9009D
:1071A000B70007002B00320050002000CE0007007F
:1071B000B600070027003A0050002000CA00070070
:1071C000B200070023003A0050002000C60007006C
:1071D000AE0007001F003A0050002000C200070068
:1071E000AA0007001B003A0050002000BE00070064
:1071F000A600070017003A0050002000BA00070060
:10720000A200070013003A0050002000B60007005B
:107210009E0007000F003A0050002000B200070057
:107220009A0007000B003A0050002000AE00070053
:107230009600070007003A0050002000AA0007004F
:107240009200070003003A0093000700C0052900E0
:1072500087ED07004F03BE004F02BE004F01BE0086
:107260004F00BE003600F900004006003600F8006E
:10727000809FBE00829FBE00849FBE00869FBE008E
:1072800087A0A9007E0007002B00320050002000DC
:10729000950007007D00070027003A0050002000FD
:1072A000910007007900070023003A0050002000F9
:1072B0008D000700750007001F003A0050002000F5
:1072C00089000700710007001B003A0050002000F1
:1072D000850007006D00070017003A0050002000ED
:1072E000810007006900070013003A0050002000E9
:1072F0007D000700650007000F003A0050002000E5
:1073000079000700610007000B003A0050002000E0
:10731000750007005D00070007003A0050002000DC
:10732000710007005900070003003A005A000700E7
:10733000900629004EED07004F03BE004F02BE002D
:107340004F01BE004F00BE003600F90000400600AD
:107350003600F800809FBE00829FBE00849FBE0062
:10736000869FBE008AA0A9006007290040ED0700A3
:107370004F03BE004F02BE004F01BE004F00BE00D3
:107380003600F900004006003600F800809FBE007D
:10739000829FBE00849FBE00869FBE008AC0A90057
:1073A0003008290032ED07004F03BE004F02BE0037
:1073B0004F01BE004F00BE003600F900004006003D
:1073C0003600F800809FBE00829FBE00849FBE00F2
:1073D000869FBE008660A9000009290024ED0700F1
:1073E0004F03BE004F02BE004F01BE004F00BE0063
:1073F0003600F90000400600809FBE008B20A900E7
:10740000CBC2BF000000D100610060000004A200F8
:1074100000404000B12C2000914078000114A100F0
:1074200080C0700001007800CBE2B700E06D800002
:10743000B00E8800C06D8000D00E8800C84DA80036
:107440004F00BE000040060085C0A90000400600B5
:107450008480A900004006008700A90000400600C3
:107460008880A900004006008C20A9002222A900E3
:10747000004006008C40A9003222A900004006000E
:10748000D4C2BF000008A30000000600D5C2BF00A0
:107490000008A30000000600BC2DEF00E06D800096
:1074A000B00E8800B82DEF00C06D8000D00E8800AF
:1074B000CB62A900CACDA80000000600D5C2BF005B
:1074C0000018A30000000600E0C2BF000068A3008F
:1074D0000000060080007800B42DEF0017040700BC
:1074E000FEFF3900000006000001E90001003A003B
:1074F000000006000200E9006700600000000000D4
:1075000011002000828F5000F9FF32000000E000DF
:107510001C003200810F500016003200E20F5000B4
:1075200012003200E30F50000E003200E40F500052
:107530000A003200E50F500006003200E60F50004E
:1075400002003200000000002100200000000000C6
:107550008100E800000000008100E8000000000059
:107560008100E800000000008100E8000000000049
:107570008100E800000000008100E800828F5000D8
:10758000DBFF3200000000000100E8000000000006
:1075900000000000000000000000000000000000EB
:1075A0000000000000000000E7004000828F500053
:1075B000CFFF3200000000000100E80000000000E2
:1075C00000000000000000000000000000000000BB
:1075D0000000000000000000E7004000828F500023
:1075E000E8FF3A00C2FF37008000780080A923003E
:1075F000808F500009003C00D30307000A003400CC
:10760000DC62A800D30307000C003200E24F5000F8
:107610000A003200B4030700000006008000780072
:10762000DC62A800F7FF3700DC62A9008000EB00F5
:107630005ACDBF00E14F5000F4FF3A00E16D8800E1
:10764000C16D8800E06D8000B00E8800C06D8000C4
:10765000D00E880000000600F0FF3700E6874700E4
:10766000889FBE008A9FBE008C9FBE008E1F780040
:10767000A86DEC00A8CDBF00FD4F50000100360002
:10768000A86DEF00A8CDBF000080FB000000400007
:10769000A1D62000F26A800002B078006066B800CF
:1076A0000000EB00F0B79F008104780039047800F7
:1076B00009077800AA03070035003500AC0307006E
:1076C0007FB197000201E80082BF9F001904780093
:1076D0008E84E800A20307003D003500A9030700DF
:1076E000E40447009E03070046003500A503070099
:1076F000E60447009A0307004F003500C403070063
:107700000006BE0019047800E8044700940307004F
:1077100011003500960307000006BE000FB8970061
:1077200064004000F0B79F00FE0F5000DFFF3A00FA
:1077300002002000031F24000A00BE00C7E3070068
:107740004F0778004F06BE004F05BE004F04BE0035
:107750006F00B10000000600020020000378240042
:1077600001E407000001BE000C00BE00FEE30700BC
:107770000005BE000006BE000FB897006400400080
:10778000F0B79F00FE0F5000C8FF3A00E8FF370037
:107790000200200003782400F3E307000001BE008C
:1077A0000C00BE00F0E307000005BE007FB19700AB
:1077B0000201E80082BF9F00190478008E84E8006F
:1077C0006140B90045E407000800E000C3FF3D0048
:1077D0000200200003782400E3E307000001BE005C
:1077E0000A00BE00E0E307000005BE0019047800AF
:1077F000E40447006140B90038E407000800E000F5
:10780000BAFF3D000200200003782400D6E3070001
:107810000001BE000A00BE00D3E307000005BE0061
:1078200019047800E60447006140B9002BE4070022
:107830000800E000B1FF3D000200200003782400B2
:10784000C9E307000001BE000A00BE00C6E307004E
:107850000006BE0019047800E80447006140B90042
:107860001EE407000800E000AAFF3D00BAFF370051
:107870004803070001003600AE2DEF0000000600AF
:10788000F06D8000E20320000280B900706A880079
:1078900000000600006E8000FAFF37008001E9005A
:1078A0000002EB00848F5000350032000300E0003E
:1078B000300032000300E9006700600000000000B3
:1078C00012002000828F51002A0032000000E000E8
:1078D0001C003200820F500016003200E20F5000F0
:1078E00012003200E30F50000E003200E40F50008F
:1078F0000A003200E50F500006003200E60F50008B
:107900000200320000000000220020000000000001
:107910000201E800000000000201E8000000000091
:107920000201E800000000000201E8000000000081
:107930000201E800000000000201E800828F51000F
:107940000C003200000000000200E800000000000F
:107950000000000000000000000000000000000027
:10796000000000000000000067014000828F51000D
:10797000F4FF3A000402E800848F5000CBFF3A0085
:10798000000006003FF50700E922A8000000000003
:10799000E922A90000000600E6C2BF000038A300EB
:1079A00001003A00B6FF3700BAFF3700FE020700B9
:1079B00002003A00CA02070000000600006E8000C4
:1079C000E20320000280B900706A8800CA0DA80096
:1079D000CA6DA900CA8DA900CAADA90000000600A1
:1079E000F6FF3700616A8000C012200026070700FA
:1079F000A802070009003C00D30207000A00340077
:107A0000DC62A800D30207000C003200E24F5000F5
:107A10000A003200E902070000000600800078003A
:107A2000DC62A800F7FF3700DC62A9008000EB00F1
:107A30005ACDBF00E14F5000F4FF3A00E16D8800DD
:107A4000C16D8800E06D8000B00E8800C06D8000C0
:107A5000D00E88005A6DEF0000000600EFFF3700DF
:107A6000D90207000E003C004C2DEC008C020700F0
:107A700008003C00B40207000B003400DC62A800E0
:107A8000B40207000D003200E24F50000B0032003C
:107A9000E0FE370080007800DC62A800F8FF3700C5
:107AA0004C2DED00F1FF3700DC62A9008000EB00F7
:107AB0005ACDBF00E14F5000F3FF3A00E16D88005E
:107AC000C16D8800E06D8000B00E8800C06D800040
:107AD000D00E880000000600EEFF3700E687470062
:107AE000889FBE008A9FBE008C9FBE008E1F7800BC
:107AF000C88DA900A86DEC00A8CDBF00FD4F5000B7
:107B000001003600A86DEF00A8CDBF000080FB008B
:107B100000004000A1D62000F26A800002B0780088
:107B20006066B8000000EB00F0B79F0081047800A9
:107B300039047800090778006140B90067E307005D
:107B40000800E000A20035000001BE000C00BE00ED
:107B500005E307000005BE007FB197000201E800C1
:107B600082BF9F00190478008E84E8006140B9004C
:107B70005AE307000800E000A50035000001BE0040
:107B80000A00BE00F8E207000005BE0019047800F4
:107B9000E40447006140B90050E307000800E0003A
:107BA000A80035000001BE000A00BE00EEE207009A
:107BB0000005BE0019047800E60447006140B900E2
:107BC00046E307000800E000AB0035000001BE00FE
:107BD0000A00BE00E4E207000006BE0019047800B7
:107BE000E80447006140B9003CE307000800E000FA
:107BF000690035000001BE000C00BE00DAE207009B
:107C00000005BE000006BE000FB8970064004000EB
:107C1000F0B79F00FE0F5000C5FF3A00E2012000C0
:107C2000F2B79F0002002000031F24000A00BE00DC
:107C30008AE20700306B8800416B8800306B80005F
:107C4000416B800002002800933824004EE30700B7
:107C50000000E000A4003D00306B8000416B80001C
:107C6000020020007338240047E307000000E00012
:107C70008F003D00306B8000416B800002002800C7
:107C80004338240040E307000000E000C0003D004E
:107C9000306B8000416B80000200200023382400FC
:107CA00039E307000000E000C7003D00306B8000B2
:107CB000416B800002002000F337240032E307000C
:107CC0000000E00096003D00306B8000416B8000BA
:107CD00002002000A33724002BE307000000E0008F
:107CE000C7003D00306B8000416B80000200200027
:107CF0000337240024E307000000E000CE003D002D
:107D0000306B8000416B800002002000633624004D
:107D10001DE307000000E0008F003D00306B800095
:107D2000416B800002002000C335240016E30700E9
:107D30000000E00088003D00CAE2A800A00020008A
:107D4000C06A880000C0EB0049F40700642DEC0015
:107D5000206B8000FD0F500005003400CAE2A8002F
:107D600040062000C06A88007FB09700206B880022
:107D700044F40700E922A80000000000E922A9005D
:107D80004F0778004F06BE004F05BE004F04BE00EF
:107D90006F00B100000006000200200003782400FC
:107DA00071E207000001BE000C00BE006EE2070099
:107DB0000005BE000006BE000FB89700640040003A
:107DC000F0B79F00FE0F500059FF3A0093FF3700B5
:107DD000020020000378240063E207000001BE00D7
:107DE0000C00BE0060E207000005BE007FB19700F6
:107DF0000201E80082BF9F00190478008E84E80029
:107E00006140B900B5E207000800E0005BFF3D00FB
:107E1000020020000378240053E207000001BE00A6
:107E20000A00BE0050E207000005BE0019047800F9
:107E3000E40447006140B900A8E207000800E00040
:107E400058FF3D00020020000378240046E20700AE
:107E50000001BE000A00BE0043E207000005BE00AC
:107E600019047800E60447006140B9009BE207006E
:107E70000800E00055FF3D000200200003782400C8
:107E800039E207000001BE000A00BE0036E207002A
:107E90000006BE0019047800E80447006140B900FC
:107EA0008EE207000800E00052FF3D00BAFF3700F5
:107EB00000C8B300EEF30700642DEF00F1F30700F4
:107EC000E922A80000000000E922A9004F0778007D
:107ED0004F06BE004F05BE004F04BE006F00B1004C
:107EE00000000600ACFF37000040EB00E0F30700A5
:107EF000642DEF00E3F30700E922A8000000000072
:107F0000E922A9004F0778004F06BE004F05BE00CA
:107F10004F04BE006F00B100000006009EFF370056
:107F200000CFB300D2F30700642DEF00D5F30700B4
:107F3000E922A80000000000E922A9004F0778000C
:107F40004F06BE004F05BE004F04BE006F00B100DB
:107F50000000060090FF3700E0CFB300C4F3070035
:107F6000642DEF00C7F30700E922A800000000001D
:107F7000E922A9004F0778004F06BE004F05BE005A
:107F80004F04BE006F00B1000000060082FF370002
:107F900000CCB300B6F30700642DEF00B9F307007F
:107FA000E922A80000000000E922A9004F0778009C
:107FB0004F06BE004F05BE004F04BE006F00B1006B
:107FC0000000060074FF370000CEB300A8F30700DE
:107FD000642DEF00ABF30700E922A80000000000C9
:107FE000E922A9004F0778004F06BE004F05BE00EA
:107FF0004F04BE006F00B1000000060066FF3700AE
:1080000080CFB3009AF30700642DEF009DF30700C3
:10801000E922A80000000000E922A9004F0778002B
:108020004F06BE004F05BE004F04BE006F00B100FA
:108030000000060058FF3700C0CFB3008CF30700E4
:10804000642DEF008FF30700E922A8000000000074
:10805000E922A9004F0778004F06BE004F05BE0079
:108060004F04BE006F00B100000006004AFF370059
:108070005A010700C9C2BF000058A3000300320024
:10808000D5C2BF000028A30007003A00CA2DA800EF
:10809000CA4DA900B42DEF00710C20002701070084
:1080A000FEFF36000000060019C8BF000008A3004C
:1080B000F6FF3A0019C8BF000028A300F3FF3A00FA
:1080C000CA4DE20031003500480107002F003A0098
:1080D00010C0B3005AEDB700DC02A900DC82A80092
:1080E0003101070050003A0043010700CA4DE20089
:1080F0004F0035003D0107004D003A00116E800031
:10810000506D8000808F50002F003900C9C2BF0021
:108110000058A30041003200D5C2BF000028A300D0
:108120003E00320019C8BF000008A3003B003A001F
:1081300019C8BF000028A30038003A001CC8BF00BF
:108140000038A30022003A00C8CDBF000028A300D9
:10815000E6FF32001C01070019003C004C2DEC002A
:10816000CF00070011003C00F700070010003C00A2
:1081700024010700F70007000F003200E24F500013
:108180000D003200D8000700D8FF3700CA8DA800C4
:10819000B42DEF0031062000E8000700C1FF3E00CB
:1081A000E6000700FCFF3600BEFF370080007800C5
:1081B000DC62A800EFFF3700DD000700CBFF3700CF
:1081C0004C2DED00E6FF3700CA000700CA8DA8005D
:1081D000616A8000C01220002B050700AD00070077
:1081E00009003C00D800070008003C00050107001A
:1081F000D800070007003200E24F500005003200AF
:10820000EE0007000000060080007800DC62A80095
:10821000F7FF3700BA000700FAFF3700CA2DA800A1
:10822000CA4DA900EAFF3700B8000700AFFF3700CA
:10823000A7000700CA8DA800E5FF3700E700070088
:10824000C942E20003003D00D5C2BF000038A300D0
:1082500007003A00CA4DA800CA2DA900B42DEF00AE
:10826000710C2000B5000700FEFF3600000006007C
:1082700019C8BF000018A300F6FF3A0019C8BF00D4
:108280000038A300F3FF3A00CA4DE2003000350089
:10829000D60007002E003A0020C0B3005AEDB70008
:1082A000DC02A800DC82A900BF0007004F003A00F2
:1082B000D1000700CA4DE2004E003500CB00070098
:1082C0004C003A00116E8000506D8000808F50008D
:1082D0002E003900C942E20041003D00D5C2BF0076
:1082E0000038A3003E00320019C8BF000018A300E8
:1082F0003B003A0019C8BF000038A30038003A001C
:108300001CC8BF000038A30022003A00C8CDBF003F
:108310000028A300E7FF3200AB00070019003C0073
:108320004C2DEC005E00070011003C0086000700A9
:1083300010003C00B3000700860007000F00320069
:10834000E24F50000D00320067000700D9FF3700F0
:10835000CAADA800B42DEF00310620007700070059
:10836000C2FF3E0075000700FCFF3600BFFF37006C
:1083700080007800DC62A800EFFF37006C00070087
:10838000CCFF37004C2DED00E6FF37005900070009
:10839000CAADA800616A8000C0122000BA040700BC
:1083A0003C00070009003C006700070008003C0093
:1083B000940007006700070007003200E24F5000FA
:1083C000050032007D0007000000060080007800F4
:1083D000DC62A800F7FF370049000700FAFF37000A
:1083E000CA4DA800CA2DA900EAFF370047000700C0
:1083F000B0FF370036000700CAADA800E5FF370020
:108400007600070040E907001CC8BF000008A30071
:1084100012003A001CC8BF000018A30013003A0065
:10842000C8CDBF000018A30014003A00C8CDBF009B
:108430000048A30015003A00C8CDBF000038A300D3
:10844000F1FF320053000700EFFF3600AE2DEF00C2
:108450001CC8BF000008A300EEFF320004FF0700A5
:108460001CC8BF000018A300EDFF320073FF070017
:10847000C8CDBF000018A300ECFF320015EF0700C5
:10848000C8CDBF000048A300EBFF320093FD0700FA
:10849000E9FF3700CA0DA9004C2DEF00C82DEF00F1
:1084A000616A800080A92300808F500000000600D0
:1084B000E20320000280B900706A8800CA0DA8009B
:1084C000CA6DA900CA8DA900CAADA90000000600A6
:1084D000CAE2A800800C2000C06A880000000600E4
:1084E000F06D8000F2FF3700BC2DEF00B82DEF00DB
:1084F0000A003700F6FF0700CA6DA800000006005A
:108500000B0007005A6DEF0000000600006E8000AF
:10851000E7FF0700AA2DEF0000000600E06D8000D5
:10852000B00E8800C06D8000D00E880000000600EC
:10853000E16D8800C16D8800F8FF3700A06D8000F4
:10854000810F50000000060010032000808F5000B3
:10855000000006005ACDBF00E14F500000000600A9
:108560006140B900DDE007000800E00000000600FF
:108570000001BE000C00BE007BE007000005BE004D
:1085800000000600220007000005BE001904780064
:1085900000000600C86DA900AE2DEC00706D8000D3
:1085A000E90F500000000600401F2000606A8800AC
:1085B000E6C2BF000038A30000000600CAFF0700A3
:1085C0005A6DEF0000000600C84DA900616A8000E6
:1085D000706A8000808F500000000600CAE2A80088
:1085E00020032000C06A880000000600CACDBF003A
:1085F0000068A30000000600B9FF0700AA2DEF00E5
:1086000000000600DC62A9008000EB00000006000C
:108610000001BE000A00BE0053E03700E023EF0077
:1086200000022200001C880020442000401C88001A
:1086300070002000501C880060042000101C88007E
:1086400000702000201C880081E3A80000000600C4
:10865000E023EF0000022000C01C8800004420003E
:10866000001D880070002000101D88007B00400065
:10867000D01C880000702000E01C880099E3A8004E
:1086800000000600C101070012E4B70012E4A800D0
:1086900013C4BF0081CFB300014060000004A000FC
:1086A00013E4B70012C4BF00014060000014A00032
:1086B00012E4B70012C4A90000000600889FBE00A3
:1086C0008A9FBE00000378000204BE000405BE00BD
:1086D0000004A80000004000000040000244200008
:1086E0008203400042B0DE00000040000242200051
:1086F0000202400043B0DE00000040008241200042
:1087000082024000E18F50001C0032004540DD0035
:10871000800B7800F07F200001002000910398007A
:10872000E3006300C208DD00F00020000100DD006E
:108730000080EA00140060008150DD00010A700032
:10874000E700630081804000300020000100DD0070
:108750000080EA00150060008158DD00810A700089
:10876000100020000600DD001424B7000004A9005A
:108770004F05BE004F04BE00000006004249DE0067
:10878000030020004511DD004048DE00010020000C
:108790006300600000014100E80B4100980398006D
:1087A000E3006300C208DD00F00020000100DD00EE
:1087B0000080EA00140060008150DD00010A7000B2
:1087C000E700630081804000300020000100DD00F0
:1087D0000080EA00150060008158DD00810A700009
:1087E000100020000600DD001424B7000004A900DA
:1087F0004F05BE004F04BE0000000600DFFF37003B
:10880000881F78008A9FBE00010478000004A80039
:1088100000004000000040000143200081024000B1
:10882000E10F52000D003200F07F200002006000D6
:1088300001002000E10F54001B0032004500DD0064
:10884000800A78000000EB00900298000004A90064
:108850004F05BE004F047800000006006115B80007
:108860004018DE0001002000630060006103B800D2
:108870004219DE00F07F20000200600001002000AD
:10888000E10F54000D0032004500DD00860A400073
:108890009A0298000004A9004F05BE004F0478001A
:1088A00000000600EDFF37004500DD00E80A40004B
:1088B0000000EB0090029800E4FF37004500DD0067
:1088C00006004000E80A40009A029800F1FF3700D5
:1088D000889FBE008A9FBE008C1F7800000678002B
:1088E0000203BE0001057800840578000100E00065
:1088F000340032004219DE00F07F200002006000E8
:108900006102B80006007800F003B2000100200008
:108910004A0CDD00C604DE00890474004A04DD0050
:108920004A39DD004630DE0000007100C638DE0046
:10893000F2FF200000036100E18F550029003200A2
:108940004229DD00CE21DE00830171004221DD00DD
:108950006150B80000007100818071000A00E000E1
:108960000C0032004462DD00027024000010A00000
:10897000003279000480E80006307900640042008B
:10898000083079004F0678004F05BE004F04BE0046
:10899000000006004462DD0002702400003279000D
:1089A0000480E80006307900640042000830790055
:1089B0004F0678004F05BE004F04BE0000000600C1
:1089C000F4FF3700F27F2000030020000600610062
:1089D0006102B8006044B80003037800E18F5500DD
:1089E000D7FF3A004229DD00CE21DE00830171006D
:1089F0004221DD006150B8000000710081807100EB
:108A00000010A0000890A000D4FF3700881F780055
:108A10004400DD00E4034000087024008883430024
:108A200006FF2F0017036300810B4300E6004000A0
:108A300082307C00E800400083307C00EA00400087
:108A400084307C006C00400005307C004F047800CE
:108A5000000006000004A800110020000008DD004E
:108A60000080EA001424B6000004A90000000600FB
:108A7000889FBE0080027800304490000880FB0090
:108A80004403DD000770240066807B00E204600080
:108A90000008A30030003A004300DD004500DE007E
:108AA00001002000A0029800B102980040C0B3006D
:108AB000A0429800E18F54004400320010C0B3007F
:108AC000904298000881FB004411DD0066004100DF
:108AD0000700400090407800814A980001F02F0084
:108AE000108060004800DE00904A98006800410055
:108AF0000700400090417800A34A98001080600071
:108B00004800DE00B04A98006A00410007004000BB
:108B100010427800C44A9800108060004800DE00CF
:108B2000D04A98006C004100070040009041780056
:108B3000E34A980090806000C808DE00F14A98007F
:108B40006401410062807B006F40600080529800A9
:108B50004F04BE0000000600C2FF210002016000B9
:108B600003002000C011DD00020020000680E800A4
:108B700060807B00F4FF2000040060000100200002
:108B8000460ADD00CA00DE00810072004600DD00FA
:108B90000201400083814800640243000702420052
:108BA00000C02F00140060004A00DE0000004100F9
:108BB000E0804900A0029800B102980030C0B300E4
:108BC000A0429800E18F5400BCFF3A0020C0B300DF
:108BD000904298004F04BE0000000600DEFF370000
:108BE000889FBE008A9FBE008C9FBE009245900069
:108BF000C85DDD001286FB00324590004855DD005F
:108C0000224490000884FB00D2449000C84CDD0050
:108C1000424390000683FB00F2439000C83BDD0016
:108C2000624190000281FB00F47F200005002000DB
:108C30000000620001002000C20EDD00CE00DE0058
:108C4000818076004200DD0000388A0015388A00F5
:108C500023388A00607024000C884500807024004E
:108C600008084500A070240006884400C070240055
:108C7000028843003064A8004F06BE004F05BE00C6
:108C80004F04BE000000060001C4BF0081CFB30046
:108C9000014060000024A00001E4B70002CEB30050
:108CA00001C8B30000C4BF0002406000814F500003
:108CB000FCFF3A003500070012E4B70012E4A800F8
:108CC00013C4BF0082CFB300024060000004A000C4
:108CD00013E4B70012C4BF00024060000014A000FB
:108CE00012E4B70012C4A90007C4BF007F406000AF
:108CF00007E4B7000004A800A0FE2F00202288008F
:108D000046A4EF0001422000F0F02F0011006000A7
:108D10000040A0000021880030FF2F001824B6007A
:108D20001424A8000004A9000004A800B0FE2F002D
:108D3000A021880036A4EF000004A90001C4BF00F0
:108D40000240600001E4B70001CEB30000C4BF00E0
:108D500001406000FDFF3A002A24EF00502180000E
:108D600040218800402180001021880010218000CF
:108D70000021880030E4A80031E4A90030C0B3002D
:108D80003064B7003164B700000006000164A80039
:108D900010C4BF00F043B20010E4B70010C4BF001D
:108DA00001CCB300014060003040B30010E4B700D4
:108DB00012C4BF00E7C04000014060008041B30022
:108DC0000000060052010700B4FA07005601070030
:108DD000B2FA07004E010700B0FA0700520107007F
:108DE000AEFA07004A010700ACFA07004E0107007F
:108DF000AAFA070046010700A8FA07004A0107007F
:108E0000A6FA070042010700A4FA0700460107007E
:108E1000A2FA37003600F800809FBE00829FBE0095
:108E2000849FBE00869FBE00300107009BFA0700AA
:108E30003D01070099FA07003501070097FA07007E
:108E40003901070095FA07003101070093FA07007E
:108E50003501070091FA07002D0107008FFA07007E
:108E6000310107008DFA0700290107008BFA07007E
:108E70002D01070089FA07004F03BE004F02BE0014
:108E80004F01BE004F00BE003600F9000040060052
:108E90003600F800809FBE00829FBE00849FBE0007
:108EA000869FBE00130107007CFA07001E01070021
:108EB0007AFA07001601070078FA07001A0107007E
:108EC00076FA07001201070074FA0700160107007E
:108ED00072FA07000E01070070FA0700120107007E
:108EE0006EFA07000A0107006CFA07000E0107007E
:108EF0006AFA07004F03BE004F02BE004F01BE00DA
:108F00004F00BE003600F900004006003600F800B1
:108F1000809FBE00829FBE00849FBE00869FBE00D1
:108F2000F60007005DFA0700FF0007005BFA070084
:108F3000F700070059FA0700FB00070057FA07007F
:108F4000F300070055FA0700F700070053FA07007F
:108F5000EF00070051FA0700F30007004FFA07007F
:108F6000EB0007004DFA0700EF0007004BFA07007F
:108F70004F03BE004F02BE004F01BE004F00BE00B7
:108F80003600F900004006003600F800809FBE0061
:108F9000829FBE00849FBE00869FBE00D90007004E
:108FA0003EFA0700E00007003CFA0700D80007007F
:108FB0003AFA0700DC00070038FA0700D40007007F
:108FC00036FA0700D800070034FA0700D00007007F
:108FD00032FA0700D400070030FA0700CC0007007F
:108FE0002EFA0700D00007002CFA07004F03BE003E
:108FF0004F02BE004F01BE004F00BE003600F90018
:10900000004006003600F800809FBE00829FBE0030
:10901000849FBE00869FBE00BC0007001FFA0700A9
:10902000C10007001DFA0700B90007001BFA07007E
:10903000BD00070019FA0700B500070017FA07007E
:10904000B900070015FA0700B100070013FA07007E
:10905000B500070011FA0700AD0007000FFA07007E
:10906000B10007000DFA07004F03BE004F02BE001B
:109070004F01BE004F00BE003600F9000040060060
:109080003600F800809FBE00829FBE00849FBE0015
:10909000869FBE009500070000FA0700A2000700A7
:1090A000FEF907009A000700FCF907009E00070080
:1090B000FAF9070096000700F8F907009A00070080
:1090C000F6F9070092000700F4F907009600070080
:1090D000F2F907008E000700F0F907009200070080
:1090E000EEF907004F03BE004F02BE004F01BE0065
:1090F0004F00BE003600F900004006003600F800C0
:10910000809FBE00829FBE00849FBE00869FBE00DF
:1091100078000700E1F9070083000700DFF9070086
:109120007B000700DDF907007F000700DBF907007F
:1091300077000700D9F907007B000700D7F907007F
:1091400073000700D5F9070077000700D3F907007F
:109150006F000700D1F9070073000700CFF907007F
:109160004F03BE004F02BE004F01BE004F00BE00C5
:109170003600F900004006003600F800809FBE006F
:10918000829FBE00849FBE00869FBE005B000700DA
:10919000C2F9070064000700C0F907005C0007007F
:1091A000BEF9070060000700BCF90700580007007F
:1091B000BAF907005C000700B8F90700540007007F
:1091C000B6F9070058000700B4F90700500007007F
:1091D000B2F9070054000700B0F907004F03BE00C2
:1091E0004F02BE004F01BE004F00BE003600F90026
:1091F000004006003600F800809FBE00829FBE003F
:10920000849FBE00869FBE003E000700A3F90700B2
:1092100045000700A1F907003D0007009FF907007E
:10922000410007009DF90700390007009BF907007E
:109230003D00070099F907003500070097F907007E
:109240003900070095F907003100070093F907007E
:109250003500070091F907004F03BE004F02BE0022
:109260004F01BE004F00BE003600F900004006006E
:109270003600F800809FBE00829FBE00849FBE0023
:10928000869FBE002100070084F907002600070022
:1092900082F907001E00070080F90700220007007E
:1092A0007EF907001A0007007CF907001E0007007E
:1092B0007AF907001600070078F907001A0007007E
:1092C00076F907001200070074F90700160007007E
:1092D00072F907004F03BE004F02BE004F01BE00EF
:1092E0004F00BE003600F900004006008020A900B3
:1092F000070037008060A900050037008040A90002
:10930000030037008080A9000100370080A0A90079
:10931000CB62A900CB82A900CAE2A80041062000C6
:109320000000EB0000000600CB62A800CB82A80082
:10933000CAE2A900410620000000EB000000060080
:10934000E40D00006600000002000000FE8EE80050
:1093500012140000028F1800120F0000068F3A004E
:10936000120F00000A8F5C00120F00000E8F7E00AB
:10937000120F0000128FAA00120F0000168FCA00F1
:10938000150F00001A8FCA00190F00001E8F32003F
:109390001A0F0000228F9A001A0F0000268F020079
:1093A0001B0F00002A8FE800121000002E8F1800FB
:1093B000120B0000328F3A00120B0000368F5C0057
:1093C000120B00003A8F7E00120B00003E8FAA00A5
:1093D000120B000000080000E4050000000000007F
:1093E000004700004000000000000000A04700000F
:1093F00060000000000000004A0E0000A000000015
:1094000002000000010000000000000000000A004F
:1094100000000000000000000064000000000000E8
:1094200000000000E8030000000000000000100041
:10943000270000000000000000A0860001000000DE
:109440000000000040420F0000000000000080000B
:1094500096980000000000000000E100F505000003
:109460000000000000CA9A003B000000000000005D
:10947000E40B5400020000000000E80076481700EA
:10948000000000000010A500D4E80000000000006B
:10949000A0724E0018090000000040007A10F3008E
:1094A0005A0000000080C600A47E8D00030000006A
:1094B00000C16F00F2862300000000008A5D780082
:1094C0004563010000006400A7B3B600E00D000092
:1094D00000E889000423C7008A000000404700001C
:1094E0002A00000002000000286E75006C6C290044
:1094F000003031003233340035363700383941001E
:1095000042434400454600003031320033343500D8
:109510003637380039616200636465006600000018
:109520006A47000026000000020000006C4792001D
:109530004700000092470900000000000200900070
:1095400047000000904706000201000000000000F4
:109550000000000000000600020200000000000001
:109560009047000006000000000000009647000041
:1095700002000000020000000100000000000000E6
:109580000EC8BF001CE8B7000FC8BF001EE8B70038
:109590001CC8BF000028A30008003200CACDBF00CD
:1095A0000068A30007003A00CB82A800CB62A800A5
:1095B000CA2DEF001AE8A800000006001AE8A9006A
:1095C00000000600DC42A900410620000000EB007C
:1095D000B2F80700DC42A800410620000000EB00C2
:1095E000AEF80700DC62A900EFFF37006800070053
:1095F000000A2000808F50000100320000000600A9
:1096000068000700C14088000000060060000700F5
:10961000000B2000808F5000010032000000060087
:1096200060000700B140880000000600889FBE006F
:10963000800478000104780009007800AAF7070088
:10964000606A8000880F500009003400080078002C
:109650004C2DB500606A8000E3F707004C0DE20076
:10966000F5FF3A00100020004F04BE000000060085
:109670004C2DEF00606A8000DBF707004C0DE20024
:10968000EDFF3A00F7FF3700889FBE008A1F780081
:1096900080047800010478000000E00001003A0036
:1096A00019002000110009000984D8000005780085
:1096B0000A00E00033003400B42DEF00A06D8000FC
:1096C000808F54001500360020032000800F5400C6
:1096D00012003400C8CDBF000028A30015003A00D6
:1096E000CA4DE2001B003500CACDBF000068A300D0
:1096F00018003A00C8CDBF000018A3001A003A00B5
:10970000C8CDBF000038A300ECFF320058F80700B6
:10971000A06D8000808F5400EBFF3E000000EB0046
:10972000B1F70700100020004F0578004F04BE007D
:1097300000000600C84DA90008007800AAF707003D
:109740008A0F54000D003C000004EB00CA4DE200FB
:10975000E5FF3D000000EB004F0578004F04BE0020
:1097600000000600F3FF37005AEA0700C8CDBF002B
:109770000038A300D1FF3200E4FF37000A04540090
:10978000D7FF37001A002000B42DEF00CBFF3700C1
:1097900009C8BF000081FB0082007800010FB20001
:1097A00000000600C810DD0008C8BF000080FB00F4
:1097B0008080400000000600FFFFFF00FFFFFF0069
:1097C000FFFFFF00FFFFFF00FFFFFF00FFFFFF00A5
:1097D000FFFFFF00FFFFFF00FFFFFF00FFFFFF0095
:1097E000FFFFFF00FFFFFF00FFFFFF00FFFFFF0085
:1097F000FFFFFF00FFFFFF00FFFFFF00FFFFFF0075
:020000040002F8
:0200000401F009
:10000000CF000000CF00000007000000A3000000A8
:10001000850000005F00000067000000C2000000D3
:10002000FF000000FF000000FF000000FF000000D4
:00000001FF
